:100000000C9499020C94CA020C94CA020C94CA0271
:100010000C94CA020C94CA020C94CA020C94CA0230
:100020000C94CA020C94CA020C94CA020C94CA0220
:100030000C94CA020C94CA020C94CA020C94CA0210
:100040000C94CA020C94CA020C94CA020C94CA0200
:100050000C94CA020C94CA020C94CA020C94B22EDC
:100060000C94CA020C94CE2F0C94A42F0C94CA02A8
:100070000C94CA020C94CA020C94CA020C94CA02D0
:100080000C94CA020C94CA020C94CA020C94CA02C0
:100090000C94CA020C94CA020C94CA020C94F82F55
:1000A0000C94CA020C94CA020C94CA020C94CA02A0
:1000B0000C94CA020C94CA020C94CA020C94CA0290
:1000C0000C94CA020C94CA020C94CA020C947A2FA3
:1000D0000C94502F0C94CA020C94262F0C94FC2ED6
:1000E0000C94CA020C94411F0C94C51F0C944F032E
:1000F0000C9454030C9421200C941A030C94111F9B
:100100000C94DD0A0C94EC1F0C94DC0A0C94AE04E5
:100110000C94B01F0C941B1F0C94070B0C941E0323
:100120000C94C32A0C94941F0C945F1F0C94122BF4
:100130000C947B1F0C941C310C9439030C943303E6
:100140000C94271F0C94DB0A0C94561F0C94221F4E
:100150000C94EF1F0C94A61F0C94E21C0C949A04B0
:100160000C94FF1E0C94D11F0C9481040C944A062D
:100170000C94851F0C94D31C0C94661F0C9447039D
:100180000C94672B0C94E61F0C9459030C947F1F5E
:100190000C94A31F0C949A1F0C94602C0C945C1F5D
:1001A0000C94002D0C94821F0C9435040C941E208A
:1001B0000C9463040C94081F0C94F0050C940B2C05
:1001C0000C94ED0A0C94591F0C94B2050C94260360
:1001D0000C94DA1F0C94141F0C9449040C94220301
:1001E0000C944B030C94431F0C9436110C94D71FA2
:1001F0000C9497060C944F1F0C94340B0C94E92C20
:100200000C9477040C94E91F0C9441030C9429037B
:100210000C94760B0C943F040C9430040C94A404BE
:100220000C94AD1F0C945B040C944E050C94DA1BDB
:100230000C94DE0A0C94481F0C942F1F0C946D0430
:100240000C9490040C94FE050C9428040C94971FB5
:100250000C94361F0C94A3050C942F030C94BC2B08
:100260000C949D1F0C94A01F0C94B8040C944B1F6D
:100270000C94E01F0C945D050C943D1F0C94E31F3F
:100280000C94D41F0C940D1F0C94691F0C94631FC5
:100290000C9455030C94DD1F0C94A81F0C941403AC
:1002A0000C94EE410C94000B0C94C2040C94391F76
:1002B0000C9453040C943D034E414E494E495459FD
:1002C000494E46CDCCCC3D0AD7233C17B7D1387721
:1002D000CC2B329595E6241FB14F0A000020410037
:1002E00000C84200401C4620BCBE4CCA1B0E5AAE81
:1002F000C59D7400407A10F35A00A0724E18090090
:1003000010A5D4E80000E87648170000E40B54027A
:100310000000CA9A3B000000E1F5050000809698B5
:1003200000000040420F000000A086010000001005
:100330002700000000E80300000000640000000047
:10034000000A00000000000100000000002C76D828
:1003500088DC674F0823DFC1DFAE59E1B1B796E50E
:10036000E3E453C63AE651997696E8E6C28426EB72
:10037000898C9B62ED407C6FFCEFBC9C9F40F2BA85
:10038000A56FA5F490055A2AF75C936B6CF9676D1D
:10039000C11BFCE0E40D47FEF520E6B500D0ED9072
:1003A0002E0300943577050080841E080000204E3F
:1003B0000A000000C80C333333330F986E128311D8
:1003C00041EF8D2114893BE65516CFFEE6DB18D1AF
:1003D000844B381BF77C1D901DA4BBE42420328481
:1003E000725E228100C9F124ECA1E53D27005EBCCC
:1003F000E2613FDD83C29C7E20A3FD1F41009D235F
:10040000BE46DB65F88C11AF32CA57E97400002193
:1004100000240027002A002D0030003300010100D5
:1004200000040107010A0100002200250028002B1A
:10043000002E003100340002010000050108010B0C
:100440000100000A0B02090C0D0E0807030401004D
:10045000000000000000000000000000000000009C
:100460000000000000000000000000000012111059
:10047000000000000000000000000000000000007C
:1004800000000000000000000020002300260029DA
:10049000002C002F003200000100000301060109BA
:1004A0000105050505070508080808020202020AF9
:1004B0000A08080404040401010101010101010307
:1004C00003030303030303040707070C0C0C0C0CC2
:1004D0000C0C0C0202020206060606060606060BB5
:1004E0000B0B0B0B0B0B0B0102102020080810202C
:1004F00040102040800201020108040201010204B0
:10050000081020408080402010080402018004026E
:1005100001804020100804020108040201010204C5
:1005200008102040800102040810204080001C3187
:10053000EE4111241FBECFEFD1E2DEBFCDBF00E000
:100540000CBF17E0A0E0B2E0EAE7FCE900E00BBF77
:1005500002C007900D92A036B107D9F72DE0A0E6B2
:10056000B7E001C01D92A73DB207E1F712E0C8E96C
:10057000D2E000E006C021970109802FFE010E9411
:10058000324AC739D10780E00807A9F70E944932EB
:100590000C942B4E0C940000FC01A089B18982E0E0
:1005A0008C93A089B1891C92A485B5851C92A685DF
:1005B000B78580E18C93108EA489B58986E08C93F1
:1005C000A289B3898C9180618C93A289B3898C9123
:1005D00088608C93A289B3898C9180688C930288FF
:1005E000F389E02D80818F7D808308958150823151
:1005F00008F05AC0E82FF0E08827EE5FFC4F8F4FDD
:100600000C94324A2203260314031A031E035403D4
:1006100029032F03330339033D03410347034B03EE
:1006200054034F0355035903809180008F778093C3
:1006300080000895809180008F7DF9CF80918000A7
:10064000877FF5CF84B58F7784BD089584B58F7D7E
:10065000FBCF8091B0008F778093B0000895809198
:10066000B0008F7DF9CF809190008F7780939000BC
:100670000895809190008F7DF9CF80919000877FC1
:10068000F5CF8091A0008F778093A000089580918E
:10069000A0008F7DF9CF8091A000877FF5CF80915A
:1006A00020018F77809320010895809120018F7D14
:1006B000F9CF80912001877FF5CFCF93DF93282F4B
:1006C00030E0F901EF5BFB4F8491F901E951FB4FF9
:1006D000D491F901EF55FB4FC491CC23A1F08111C6
:1006E0000E94F602EC2FF0E0EE0FFF1FE957FB4FE0
:1006F000A591B491EC91ED2381E090E009F480E0C4
:10070000DF91CF91089580E090E0FACF1F93CF93CF
:10071000DF93282F30E0F901EF5BFB4F8491F90163
:10072000E951FB4FD491F901EF55FB4FC491CC2314
:10073000A9F0162F81110E94F602EC2FF0E0EE0FC7
:10074000FF1FE95DFB4FA591B4918FB7F894EC9131
:10075000111108C0D095DE23DC938FBFDF91CF91BC
:100760001F910895DE2BF8CFCF93DF9390E0FC012B
:10077000E951FB4F24918F559B4FFC0184918823B5
:10078000C9F090E0880F991FFC01E35FFB4FA59132
:10079000B491FC01E95DFB4FC591D49161110DC08D
:1007A0009FB7F8948C91209582238C93888128237D
:1007B00028839FBFDF91CF910895623051F49FB796
:1007C000F8943C91822F809583238C93E8812E2B83
:1007D000EFCF8FB7F894EC912E2B2C938FBFEACFED
:1007E0001F93CF93DF93182FEB0161E00E94B403B6
:1007F000209739F460E0812FDF91CF911F910C9405
:100800008603CF3FD10511F461E0F5CFE12FF0E091
:10081000EF5BFB4FE491E150E23108F0B3C0F0E050
:100820008827EA5EFB4F8F4F0C94324A280430042D
:1008300035043F044904C20453045B0463046D049B
:100840007704810490049A04C204A404AE04B8049A
:1008500084B5806884BDC7BDDF91CF911F91089595
:1008600084B5806284BDC8BDF7CF80918000806868
:1008700080938000D0938900C0938800EDCF809151
:100880008000806280938000D0938B00C0938A00A8
:10089000E3CF80918000886080938000D0938D00AA
:1008A000C0938C00D9CF8091B00080688093B00055
:1008B000C093B300D1CF8091B00080628093B0002C
:1008C000C093B400C9CF809190008068809390005D
:1008D000D0939900C0939800BFCF80919000806220
:1008E00080939000D0939B00C0939A00B5CF8091E5
:1008F0009000886080939000D0939D00C0939C00EE
:10090000ABCF8091A00080688093A0008091A00070
:100910008F7B8093A000D093A900C093A8009CCFA8
:100920008091A00080628093A000D093AB00C09320
:10093000AA0092CF8091A00088608093A000D093FD
:10094000AD00C093AC0088CF809120018068809377
:100950002001D0932901C09328017ECF80912001EE
:10096000806280932001D0932B01C0932A0174CF21
:1009700080912001886080932001D0932D01C09345
:100980002C016ACFC038D1050CF03ECF33CF86336F
:1009900008F0865320917B00982F9870277F922B28
:1009A00090937B002091B10290E4299F9001112443
:1009B0008770822B80937C0080917A008064809382
:1009C0007A0080917A0086FDFCCF8091780090912A
:1009D000790008953FB7F8948091370B9091380BC8
:1009E000A091390BB0913A0B26B5A89B05C02F3FBB
:1009F00019F00196A11DB11D3FBFBA2FA92F982F45
:100A00008827BC01CD01620F711D811D911D42E03F
:100A1000660F771F881F991F4A95D1F708958F9207
:100A20009F92AF92BF92CF92DF92EF92FF926B01B3
:100A30007C010E94EA044B015C01C114D104E10471
:100A4000F104B9F00E94EA04681979098A099B093E
:100A5000683E73408105910580F321E0C21AD108F8
:100A6000E108F10888EE880E83E0981EA11CB11CF5
:100A7000E4CFFF90EF90DF90CF90BF90AF909F902A
:100A80008F9008952FB7F8946091330B7091340BC9
:100A90008091350B9091360B2FBF08950895DB019F
:100AA00014964D915C9115976D917C91DC01ED91BF
:100AB000FC910280F381E02D1994AF92BF92CF9206
:100AC000DF92EF92FF920F931F93CF93DF936C010E
:100AD0007B018B01040F151FEB015E01AE18BF08EF
:100AE000C017D10759F06991D601ED91FC910190A1
:100AF000F081E02DC6011995892B79F7C501DF91A9
:100B0000CF911F910F91FF90EF90DF90CF90BF900A
:100B1000AF900895FC01A089B1898C91A689B7890D
:100B200082FD0FC09C91818D8F5F8F73228D821704
:100B300049F0A18DAE0FBF2FB11D5D969C93818FA3
:100B400008958C910895FC01538D448D252F30E03C
:100B5000842F90E0821B930B541710F0CF960895CA
:100B600001970895FC01918D828D981761F0A28DF7
:100B7000AE0FBF2FB11D5D968C91928D9F5F9F73BD
:100B8000928F90E008958FEF9FEF08950F931F933A
:100B9000CF93DF93EC010E944205688779878A87AB
:100BA0009B87CE010E94B20597FF15C00E944205A7
:100BB000088519852A853B85601B710B820B930B79
:100BC0000C811D812E813F81601771078207930779
:100BD00040F38FEF9FEFDF91CF911F910F91089519
:100BE000FC01918D828D981731F0828DE80FF11DF7
:100BF000858D90E008958FEF9FEF0895FC01918D12
:100C0000228D892F90E0805C9F4F821B91098F730A
:100C10009927089583E99BE00E94FE0521E0892B36
:100C200009F420E0822F089580E39CE00E94FE05F5
:100C300021E0892B09F420E0822F08958DEC9CE0BF
:100C40000E94FE0521E0892B09F420E0822F0895FF
:100C5000FC01A48DA80FB92FB11DA35ABF4F2C9131
:100C6000848D90E001968F739927848FA689B78928
:100C70002C93A089B1898C91837080648C93938D1F
:100C8000848D981306C00288F389E02D80818F7DC2
:100C900080830895EF92FF920F931F93CF93DF937A
:100CA000EC0181E0888F9B8D8C8D98131AC0E889A8
:100CB000F989808185FF15C09FB7F894EE89FF8977
:100CC0006083E889F98980818370806480839FBF15
:100CD00081E090E0DF91CF911F910F91FF90EF9015
:100CE0000895F62E0B8D10E00F5F1F4F0F73112725
:100CF000E02E8C8D8E110CC00FB607FCFACFE88960
:100D0000F989808185FFF5CFCE010E942806F1CFB9
:100D1000EB8DEC0FFD2FF11DE35AFF4FF0829FB7D3
:100D2000F8940B8FEA89FB8980818062CFCFCF93C3
:100D3000DF93EC01888D8823B9F0AA89BB89E88903
:100D4000F9898C9185FD03C0808186FD0DC00FB6A9
:100D500007FCF7CF8C9185FFF2CF808185FFEDCF27
:100D6000CE010E942806E9CFDF91CF91089580E05F
:100D700090E0892B29F00E941E0681110E9400003C
:100D800080E090E0892B49F080E090E0892B29F009
:100D90000E94000081110E94000080E090E0892BF9
:100DA00029F00E94140681110E94000080E090E06A
:100DB000892B29F00E940A0681110C9400000895E5
:100DC000CF92DF92EF92FF920F931F93CF93DF9317
:100DD0007C016B01EA01DC01ED91FC9161E0808115
:100DE0000E94860301E811E0C09EC001C19E900DE3
:100DF000D09E900D1124880F991F880F991F059779
:100E00000197F1F7D701ED91FC9160E080810E949C
:100E10008603C09FC001C19F900DD09F900D1124EB
:100E2000880F991F880F991F05970197F1F7DF9198
:100E3000CF911F910F91FF90EF90DF90CF90089589
:100E4000DC0180E0615090F09D919827E92FEF70D0
:100E5000F0E0E351FC4F2491E92FE295EF70F0E0D0
:100E6000E350FC4FE491822F8E27ECCF0895DC01F4
:100E70002C911196ED91FC91F8948181822B8183C4
:100E80009281322F30959323928387E090E00197EF
:100E9000F1F781818323818383E290E00197F1F769
:100EA00090817894EFECF0E03197F1F7922381E0B4
:100EB00009F480E00895FC0190810180F281E02D29
:100EC000292F209560FF14C0F894828182238283A9
:100ED0008181892B8183A3E2B0E01197F1F78281B0
:100EE000982B9283789487ED90E00197F1F708951D
:100EF000F8948281822382838181892B8183AFEF61
:100F0000B0E01197F1F78281982B928378948FE06B
:100F100090E0EBCFDF92EF92FF920F931F93CF936E
:100F2000DF93EC01D62EE42E08E010E0FF24F394CA
:100F300061E08D2D8F2109F460E0CE010E945B07F6
:100F4000FF0C01501109A1F7E11010C0F894E981DC
:100F5000FA8191818881809589238183E981FA8151
:100F6000928188818095892382837894DF91CF91C3
:100F70001F910F91FF90EF90DF900895EF92FF92F5
:100F80000F931F93CF93DF938C017B0140E065E5C6
:100F90000E948A07E70188E0E80EF11C699140E0B1
:100FA000C8010E948A07CE15DF05C1F7DF91CF91F6
:100FB0001F910F91FF90EF900895FC0190810180A7
:100FC000F281E02DF8948181292F2095822381835D
:100FD00078943DE743E050E0315029F1DA01119770
:100FE000F1F780818923C1F3F8948281822382837F
:100FF0008181892B81837894ABE7B7E01197F1F772
:10100000F894818182238183A3E1B1E01197F1F704
:101010008081982381E009F080E07894E3E6F6E0AF
:101020003197F1F7089580E008956F927F928F9243
:101030009F92AF92BF92CF92DF92EF92FF920F9367
:101040001F93CF93DF938C01EB018091B50D9091AD
:10105000B60D0E94DD07882309F43FC0B8018091D6
:10106000B50D9091B60D0E94BE0740E06EEB8091E9
:10107000B50D9091B60D0E948A077E016E0189E040
:10108000C80ED11C8E01A090B50DB090B60D88E0B1
:10109000882E912C712C66246394C5010E94370719
:1010A00081117628660CE1E08E1A9108B1F7F801FB
:1010B00071928F01CE16DF0631F78091B50D9091B8
:1010C000B60D0E94DD07813041F4F70181917F0167
:1010D000811105C0E017F107C1F790E008C068E092
:1010E000CE010E94200791E028852813F6CF892F92
:1010F000DF91CF911F910F91FF90EF90DF90CF90F4
:10110000BF90AF909F908F907F906F900895CF93F6
:10111000DF9300D000D000D0CDB7DEB7BE016F5F47
:101120007F4F8BE39BE00E941508811105C060E0B2
:1011300070E08EEF92EC3EC06A8170E0762F6627F9
:10114000770F770F770F298148E0249F90011124B2
:10115000262B372B80913B0B8031E1F46885662389
:10116000C9F070E08F81AB01481B5109CA01969507
:10117000982F8827979587950E941E4ACB018097C4
:10118000B90153E0660F771F5A95E1F760789C012B
:10119000260F371F213854EE35074CF2B901330FB3
:1011A000880B990B0E94734720E030E040E05CE33D
:1011B0000E94D24729960FB6F894DEBF0FBECDBF6E
:1011C000DF91CF910895CF93DF9300D000D000D06E
:1011D000CDB7DEB7BE016F5F7F4F0E941508882331
:1011E00031F08D818F33A9F020F48F31A1F080E0B0
:1011F00007C08F3521F08F37D1F78CE001C08BE02D
:1012000029960FB6F894DEBF0FBECDBFDF91CF9108
:1012100008958AE0F5CF89E0F3CFCF92DF92EF9285
:10122000FF92CF9380913B0B803159F18BE39BE090
:101230000E94E308C82F882309F46EC08091B50D81
:101240009091B60D0E94DD076BE37BE08091B50DB8
:101250009091B60D0E94BE074091AC0D64E4809160
:10126000B50D9091B60D0E948A078091B00D811145
:101270000AC0C1E08C2FCF91FF90EF90DF90CF900C
:101280000895CCE0DBCF8091B10D8823E1F080910F
:10129000AC0D811118C00E9442056B017C01809148
:1012A000B50D9091B60D0E943707813011F30E9461
:1012B00042056C197D098E099F096E3E72408105B9
:1012C000910568F3D6CFC9508EEE92E0C33040F45A
:1012D000EC2FF0E0EE0FFF1FE35CFC4F808191816B
:1012E0006C01990FEE08FF088091AD0D882329F05D
:1012F00060E08091AE0D0E948603C701B6010E9496
:101300000F05C091AD0DCC2309F4B3CF61E08091FE
:10131000AE0D0E948603AECFC0E0ACCF2091DC07BB
:10132000260F3327331F21323105ECF42091690B4E
:10133000FC0190E080E0243069F082E00895A09103
:10134000DC072191AC014654584FA40FB52FB11DB5
:101350002C930196861798F38091DC07680F6093B1
:10136000DC0780E0089581E008951092690B81E028
:101370008093680B1092430B61E084E10E94860326
:1013800061E085E10E948603E9EBF0E080818E7FD9
:10139000808380818D7F808388E48093B80085E49A
:1013A0008093BC000895CF93DF9391E09093B907A9
:1013B0008823B9F0C091B800D091BA008091BC00E8
:1013C0008A7B8093BC0060E084E10E94860360E039
:1013D00085E10E9486030E94B509D093BA00C093AC
:1013E000B800DF91CF910895CF92DF92EF92FF92F4
:1013F0000F931F93CF93DF93D091920B81E0D13263
:1014000008F09CC0C091910B0E94EA046B017C0122
:101410008091690B81116CC082E08093690B81E03F
:101420008093680B8FEF8093670B1092660BD093BD
:10143000650BA1E7BBE0E5E4FBE080E0D8138DC0DD
:101440001092440B8091440BCC0FC82BC093440BDB
:101450008091430B813009F084C01092430B0E94AD
:10146000EA046B017C018091440B8093BB00809166
:101470006B0B90916C0BA0916D0BB0916E0B892B47
:101480008A2B8B2BA1F00E94EA0400916B0B109128
:101490006C0B20916D0B30916E0B6C197D098E09D0
:1014A0009F09061717072807390708F442C08091DB
:1014B000BC0083FDD8CF85EC8093BC000E94EA0479
:1014C0006B017C018091690B823009F44CC08091E2
:1014D000670B8F3F09F469C08091670B803209F474
:1014E00066C08091670B803309F463C084E026C036
:1014F00080916B0B90916C0BA0916D0BB0916E0B6A
:10150000892B8A2B8B2B09F483CF0E94EA0400914C
:101510006B0B10916C0B20916D0B30916E0B6C1955
:101520007D098E099F09061717072807390708F054
:101530006FCF80916A0B0E94D30985E01092700BE7
:101540001092920B10926F0BDF91CF911F910F9120
:10155000FF90EF90DF90CF9008959D9191938F5FD2
:101560006DCF85EEA9CF80916B0B90916C0BA09104
:101570006D0BB0916E0B892B8A2B8B2B09F4A2CFAC
:101580000E94EA0400916B0B10916C0B20916D0B83
:1015900030916E0B6C197D098E099F09061717078C
:1015A0002807390708F08ECFC4CF80E0C7CF82E08C
:1015B000C5CF83E0C3CF089508950895E091B8079B
:1015C0008091B707E81730F4F0E0E956F84F8081D2
:1015D00090E008958FEF9FEF08959091B807809164
:1015E000B7072FEF3FEF981748F4E92FF0E0E956DF
:1015F000F84F208130E09F5F9093B807C9010895AC
:101600008091B7079091B807891B990B0895CF92E5
:10161000DF92EF92FF920F931F93CF93DF937C01A2
:10162000CB018A0120916F0B222389F0EB016B0122
:10163000C40ED51ECC15DD0569F06991D701ED9179
:10164000FC910190F081E02DC7011995F3CF642F33
:101650000E948E09C801DF91CF911F910F91FF90D9
:10166000EF90DF90CF900895CF93DF931F92CDB787
:10167000DEB7698320916F0B2223F9F02091920B42
:10168000203258F021E030E0FC013383228390E0E7
:1016900080E00F90DF91CF9108958091700BE82F3B
:1016A000F0E0EF58F44F998190838F5F8093700B37
:1016B0008093920B81E090E0ECCF61E0CE01019647
:1016C0000E948E09F7CFFC01248131E030936F0B2B
:1016D0002093910B1092700B1092920B8485682BC3
:1016E0008AE69DE00E94340B0C94F40990E080E0BF
:1016F0000895609393077093940780939507909350
:101700009607645D7E4F8F4F9F4F60938F07709356
:101710009007809391079093920782E090E09093D6
:101720008E0780938D070E9442056093890770930E
:101730008A0780938B0790938C070895CF92DF924E
:10174000EF92FF920F931F930E9442058B019C0121
:10175000C0908907D0908A07E0908B07F0908C07A3
:1017600060919307709194078091950790919607E7
:101770000C191D092E093F09083E134021053105AA
:10178000E0F0DC01CB010196A11DB11D8093930710
:1017900090939407A0939507B0939607B701A6017D
:1017A00048515C4F6F4F7F4F4093890750938A0792
:1017B00060938B0770938C07C7CF1F910F91FF9099
:1017C000EF90DF90CF9008954F925F926F927F924B
:1017D0008F929F92AF92BF92CF92DF92EF92FF9241
:1017E0000F931F93CF93DF934B015C0180917E0792
:1017F00090917F07A0918007B09181078815990586
:10180000AA05BB0509F4C6C08CE3C82ED12CE12C77
:10181000F12CC501A70196010E94D348609382076D
:10182000CA01B901A70196010E94D34860938307BA
:10183000C501B40120E13EE040E050E00E94D34801
:10184000CA01B90128E130E040E050E00E94D348ED
:1018500060938407C501B40120E831E541E050E020
:101860000E94D34869017A01CA01B9016C5F7F4FB8
:101870008F4F9F4F27E030E040E050E00E94D34878
:101880006F5F60938507412C512C320140E004E6E4
:1018900010E0C0E9D1E0242F30E02E54384FF90198
:1018A000E370FF273097F9F4C901B8010E941E4A7E
:1018B000892B31F4C901BE010E941E4A892B99F47B
:1018C0008EE691E0A0E0B0E0480E591E6A1E7B1E35
:1018D000D301C201AA27BB27C816D906EA06FB0610
:1018E00038F04F5FD8CF8DE691E0A0E0B0E0ECCFCC
:1018F00040938807C90164E670E00E941E4AEC012B
:10190000C90160E971E00E941E4A309721F42097D6
:10191000D9F40097C9F04DE651E060E070E0441A58
:10192000550A660A770AC418D508E608F708A1E33D
:10193000B3E020E0213069F43097E9F5209711F405
:101940000097C9F54DE106C04EE651E060E070E059
:10195000E6CF4C9150E070E060E031E0320FC41609
:10196000D506E606F70640F0C41AD50AE60AF70AD5
:101970001196232F3C30F1F62F5F20938707C394F5
:10198000C092860780927E0790927F07A092800780
:10199000B0928107DF91CF911F910F91FF90EF904F
:1019A000DF90CF90BF90AF909F908F907F906F907F
:1019B0005F904F9008954CE1CDCF0E949E0B0E9406
:1019C000E40B8091820790E008950E949E0B0E9494
:1019D000E40B8091830790E008950E949E0B0E9483
:1019E000E40B8091840790E008951F93CF93DF93D9
:1019F000182F0E94C704EC01812F0E94C704BE016A
:101A0000680F791F072E000C880B990B0E947347F3
:101A100020E030E040E05FE30E94D247DF91CF91C9
:101A20001F91089580913802882341F088E08093C7
:101A3000A70D60E08BE99DE00C94630B88E0809338
:101A40009A0D60E08EE89DE0F7CFBC0180913802EE
:101A5000882321F08BE99DE00C944F058EE89DE0F2
:101A6000FBCFAF92BF92CF92DF92EF92FF921F9384
:101A7000CF93DF93CDB7DEB7A4970FB6F894DEBF50
:101A80000FBECDBF90915608992309F452C0182F6C
:101A900080913B02811709F448C08CE797E09CA332
:101AA0008BA382E2E3E7F3E0DE01119601900D9251
:101AB0008A95E1F781E38E8B8D8B8E8F8D8F81E3FD
:101AC000111101C080E3888F81E3111180E388A3A5
:101AD0008FE0E82EF12C5E0181E2A80EB11CFE0120
:101AE00031966F01F60181916F0142E050E061E0B3
:101AF00070E0813321F441E050E062E070E0CE011B
:101B000083960E94E006AC14BD0461F741E150E009
:101B100061E070E0CE0183960E94E006F1E0EF1AEA
:101B2000F108E9F610933B0204C00E94E50C80FF27
:101B3000B4CFA4960FB6F894DEBF0FBECDBFDF9131
:101B4000CF911F91FF90EF90DF90CF90BF90AF901B
:101B50000895CF92DF92EF92FF92CF93DF9310928E
:101B60003A021092390280916607882309F448C02E
:101B700020E030E048E452E46091E8027091E9022C
:101B80008091EA029091EB020E94044920E030E04B
:101B900040EA50E40E9471490E94E3496B0161E010
:101BA0008EE30E9486036FEF70E088E00E94F003EE
:101BB000D7FE04C0D0923A02C09239028091390215
:101BC00090913A02029734F482E090E090933A02C6
:101BD00080933902809165078823E1F060E08FE30C
:101BE0000E94860360E080E40E9486036FEF8AE033
:101BF000DF91CF91FF90EF90DF90CF900C94860310
:101C000060E08EE30E94860370E060E088E00E945E
:101C1000F003E0CF61E08FE30E94860361E080E49F
:101C20000E94860370E060E08AE0DF91CF91FF9030
:101C3000EF90DF90CF900C94F003CF930E94DD0CD7
:101C400020916207309163078217930709F442C01D
:101C5000C1E0C09367070E94DD0C9C01909363076D
:101C60008093620765E070E00E941E4A892B11F4A0
:101C7000C0936807C9016AE070E00E941E4A892B80
:101C800019F481E080936907C9016FE070E00E9458
:101C90001E4A892B19F481E080936A07C9016EE11D
:101CA00070E00E941E4A892B19F481E080936B0733
:101CB0000E94E50C2091600730916107821793071D
:101CC00049F081E080936C070E94E50C90936107D6
:101CD00080936007CF910895CF93DF9385E40E94AE
:101CE0005D03EC0181E0209709F080E08093C30A56
:101CF00084E40E945D039C0181E02115310509F017
:101D000080E08093C20ACD2B19F091E0232B09F4D7
:101D100090E09093BD0A8091C50A882391F083E4F6
:101D20000E945D0321E0892B09F020E020935708F1
:101D300082E40E945D0321E0892B09F020E02093DA
:101D40005508DF91CF91089581E080935608109255
:101D50003B020E94310D68EE73E080E090E00E944B
:101D60000F0580E00E94310D68EE73E080E090E0A6
:101D70000E940F0581E00E94310D68EE73E080E063
:101D800090E00E940F0580E00E94310D10925608ED
:101D900008958F929F92AF92BF92CF92DF92EF926F
:101DA000FF921092150810921408109217081092C2
:101DB0001608109219081092180810928E021092AC
:101DC0008F02109290021092910210929202109241
:101DD0009302109294021092950210926B0210924C
:101DE0006C0210926D0210926E0210926F021092AD
:101DF00070021092710210927202109248021092B8
:101E0000490210924A0210924B0210924C02109218
:101E10004D0210924E0210924F0281EF9FEF90936D
:101E2000080B8093070B8091C20A882341F08091B0
:101E3000F4029091F5029093F7028093F6021092CB
:101E4000E80A10921F088090E8029090E902A090A2
:101E5000EA02B090EB026091F2027091F302072E59
:101E6000000C880B990B0E9473476B017C01AC013D
:101E70009B01C501B4010E94194A87FD0DC0109253
:101E8000F7021092F602FF90EF90DF90CF90BF9094
:101E9000AF909F908F9008958091F4029091F502F9
:101EA00047972091F6023091F702281739073CF046
:101EB00080916407811103C081E080931F088091A5
:101EC0001F08882301F3A7019601C501B4010E94F0
:101ED0006C471816C4F281E08093E80AA5019401CA
:101EE000C701B6010E94044920E030E04AE754E40B
:101EF0000E94D24720E030E04AE754E40E940549BE
:101F00000E94EA49683E83E0780710F468EE73E0C7
:101F1000693B8BE0780710F068EB7BE070930C086E
:101F200060930B08B0CFBF92CF92DF92EF92FF92F7
:101F30000F931F93CF93DF93EC01B62EC72E8D85A1
:101F4000811105C0CE010E94DD0781110EC01B86E4
:101F50001D861C8680E0DF91CF911F910F91FF902D
:101F6000EF90DF90CF90BF90089540E060EFCE01FA
:101F70000E948A0701E0E12CD12C11E0CE010E94E1
:101F80003707F82ECE010E94370791E0F91218C0EA
:101F9000813099F51134D8F2DB86D11002C081E08E
:101FA0008D878B81882399F22396EB2DFC2DCF0111
:101FB000089629912193E817F907D9F781E0CBCF4B
:101FC000EE2DF0E0F8120FC08B851817A0F4DE019B
:101FD000AE0FBF1F13968C91802379F4F12C19302A
:101FE00008F41C87D12EEC0FFD1F8381902F909554
:101FF000892383830AC08113F1CFFE01EE0DF11D09
:102000008381802B8383FF24F3946F2DCE010E9464
:102010005B071F5F000F11F4E39401E087E08E156A
:1020200008F0ACCFB7CFFF920F931F93CF93DF93FE
:102030008C01F62EE091B50DF091B60D1386158644
:1020400014861286118610861782168215821482D3
:102050001382C0E0B8018091B50D9091B60D0E9439
:10206000930FD82F882329F0FC1629F0CF5FFC1698
:1020700088F7D0E008C067E0C8010E942007F80197
:1020800097818913F3CF8D2FDF91CF911F910F91FE
:10209000FF9008950F931F93CF938C01C62F0E943A
:1020A000630B6C2F6460C8010E94630B6C2F6B7F05
:1020B000C8010E94630B83EC90E00197F1F7CF9188
:1020C0001F910F9108950F931F93CF93DF938C016E
:1020D000D62FC42F607F642B0E944A1080E1D89FC6
:1020E000B00111246C2BC801DF91CF911F910F918A
:1020F0000C944A10CF93DF9300D000D01F921F9210
:10210000CDB7DEB728E0EFEFF2E0DE0111960190E7
:102110000D922A95E1F7FC012085241710F44FEF6A
:10212000420F50E0440F551F21E030E02C0F3D1FBF
:10213000420F531FFA012081620F606840E0289629
:102140000FB6F894DEBF0FBECDBFDF91CF910C94D8
:102150006310462F90913802682F992321F08BE964
:102160009DE00C947A108EE89DE0FBCFCF93DF9337
:10217000EC0140E061E00E9463108BE39FE1019776
:10218000F1F78985882339F040E060E0CE01DF91E6
:10219000CF910C947A10DF91CF910895FF920F9315
:1021A0001F93CF93DF93EC018D8188608D8384E052
:1021B000F82EF88662E370E080E090E00E940F0560
:1021C0006C85CE010E94630B68EE73E080E090E0C6
:1021D0000E940F0560E3CE010E944A100BE416E452
:1021E000C8010197F1F760E3CE010E944A10C801CF
:1021F0000197F1F760E3CE010E944A1083E592E077
:102200000197F1F760E2CE010E944A106D81606291
:1022100040E0CE010E946310FE8240E06CE0CE01FF
:102220000E946310CE010E94B61082E08F8340E0CE
:1022300066E0CE010E94631040E062E0CE010E94A1
:1022400063108BE39FE10197F1F7DF91CF911F912D
:102250000F91FF90089580913802882321F08BE937
:102260009DE00C94B6108EE89DE0FBCF41E00E940B
:10227000631081E090E00895EF92FF920F931F9317
:10228000CF93DF938C017A0188E0689FB00111241D
:10229000606440E0C8010E946310E70188E0E80E36
:1022A000F11C6991C8010E943611CE15DF05C9F7EE
:1022B000DF91CF911F910F91FF90EF900895682FBC
:1022C00080913802882321F08BE99DE00C9436112F
:1022D0008EE89DE0FBCFFF920F931F93CF93DF9388
:1022E0000EEB12E0D0E0C0E0F801F1908F01CE01DA
:1022F0000E949348F81621F06F2DCE010E949B4852
:102300002196CA32D10581F78EEB92E0DF91CF9111
:102310001F910F91FF9008950F931F93CF93DF9319
:102320000EEB12E0D0E0C0E0CE010E949348F8012D
:1023300081938F012196CA32D105B1F764EF71E024
:1023400080E090E0DF91CF911F910F910C940F05E9
:10235000FB0101900020E9F73197AF01461B570BB5
:102360000C945D058F929F92AF92BF92CF92DF92B5
:10237000EF92FF920F931F93CF93DF93CDB7DEB70A
:10238000A1970FB6F894DEBF0FBECDBF6C01990FB9
:10239000EE08FF08F7FE4BC06DE28DEC9CE00E945A
:1023A0004A068C0122273327A9012C193D094E0921
:1023B0005F0919A2CE0181967C019AE0892E912CA9
:1023C000A12CB12CCA01B901A50194010E94D348E6
:1023D000605DF70162937F012115310541055105CB
:1023E00089F790E080E0309729F0BF018DEC9CE008
:1023F0000E94A811080F191F65E973E08DEC9CE09D
:102400000E94A811800F911FA1960FB6F894DEBF0D
:102410000FBECDBFDF91CF911F910F91FF90EF9035
:10242000DF90CF90BF90AF909F908F900895A701BD
:10243000960119A28E010F5D1F4F8AE0C82ED12C84
:10244000E12CF12CCA01B901A70196010E94D348E1
:10245000605DF80162938F01211531054105510539
:1024600089F7309739F0BF018DEC9CE00E94A811EC
:102470008C01C2CF10E000E0BFCF0F931F93CF932A
:10248000DF93EC010E94A8118C0165E973E0CE0195
:102490000E94A811800F911FDF91CF911F910F9182
:1024A0000895CF93DF93CDB7DEB7AA970FB6F89410
:1024B000DEBF0FBECDBF8AE2E7E0F3E0DE0111969A
:1024C00001900D928A95E1F78AE2FE013196AEEB1A
:1024D000B2E001900D928A95E1F768E973E08DEC26
:1024E0009CE00E943D120E946B1164EF71E080E05D
:1024F00090E0AA960FB6F894DEBF0FBECDBFDF9175
:10250000CF910C940F058091F6029091F702909371
:10251000C7028093C60267EA73E08DEC9CE00E94DC
:102520003D1268EE73E080E090E00E940F050C948D
:10253000000008950F931F93CF93DF93EC010E9447
:102540004F058C0165E973E0CE010E94A811800F50
:10255000911FDF91CF911F910F9108950F931F93BA
:10256000CF93DF938C01EB01FC0180819181009777
:10257000E1F06881798161157105A9F0428153818B
:102580002C813D814217530770F00E943F4B8C8194
:102590009D81F801958384831D821C82DF91CF91F8
:1025A0001F910F9108950E94B84288819981F80186
:1025B000918380838A819B81938382838C819D8197
:1025C00095838483198218821B821A82E5CFCF9368
:1025D000DF93EC0188819981009711F00E94B84245
:1025E000198218821D821C821B821A82DF91CF9170
:1025F0000895FC0180819181009711F00C94B842FC
:1026000008950F931F93CF93DF93EC0188819981F5
:10261000009759F02A813B812617370730F081E077
:10262000DF91CF911F910F9108958B016F5F7F4FC5
:102630000E94554A009759F0998388831B830A8327
:102640002C813D81232B59F7FC011082E8CF80E0DB
:10265000E7CFEF92FF920F931F93CF93DF93611514
:10266000710541F480E0DF91CF911F910F91FF90B0
:10267000EF90089541155105B1F07B01EC010C81FB
:102680001D81040F151FB8010E940113882351F307
:10269000288139818C819D81B701820F931F0E940F
:1026A0003F4B1D830C8381E0DECFCF93DF93EC01A2
:1026B000FB0101900020E9F73197AF01461B570B52
:1026C0000E942913811103C0CE010E94E712CE019E
:1026D000DF91CF910895CF93DF93EC01FB0144810B
:1026E0005581608171810E942913811103C0CE013F
:1026F0000E94E712CE01DF91CF910895FB01019076
:102700000020E9F73197AF01461B570B0C942913B2
:10271000FB0144815581608171810C942913EF92F2
:10272000FF920F931F93CF93DF93EC017B018A01FC
:10273000BA010E94011381110BC0CE010E94E71261
:10274000CE01DF91CF911F910F91FF90EF900895EF
:102750001D830C83B701888199810E943F4BF0CF84
:10276000FB0101900020E9F73197AF01461B570BA1
:102770000C948F130F931F93CF93DF93CDB7DEB7D6
:1027800062970FB6F894DEBF0FBECDBF8C01CB01B0
:10279000F8011182108213821282158214824AE09B
:1027A000BE016F5F7F4F0E944543BE016F5F7F4F49
:1027B000C8010E94B01362960FB6F894DEBF0FBE38
:1027C000CDBFDF91CF911F910F910895EF92FF92AE
:1027D0000F931F93CF93DF93CDB7DEB7A1970FB6BB
:1027E000F894DEBF0FBECDBF7C01CB01BA01F7016B
:1027F0001182108213821282158214828E010F5F61
:102800001F4F22E044E00E94FE41009789F0BC0186
:10281000C7010E94B013A1960FB6F894DEBF0FBE99
:10282000CDBFDF91CF911F910F91FF90EF90089551
:10283000C7010E94E712EFCF0F931F93CF93DF934F
:10284000CDB7DEB7A1970FB6F894DEBF0FBECDBFF0
:102850008C01CB01BA01F80111821082138212821D
:10286000158214822AE0AE014F5F5F4F0E945043F1
:10287000BE016F5F7F4FC8010E94B013A1960FB6D3
:10288000F894DEBF0FBECDBFDF91CF911F910F91A6
:102890000895CF93DF93EC01FB018617970749F06A
:1028A000608171816115710541F0448155810E94FB
:1028B0008F13CE01DF91CF9108950E94E712F9CFD7
:1028C000FC011182108213821282158214820C94F0
:1028D00049140F931F93CF93DF9300D000D0CDB74F
:1028E000DEB78C01862F642F70E090E00E94A91063
:1028F000B801CE0101960E946014CE0101960E949B
:10290000250DCE0101960E94F91226960FB6F89475
:10291000DEBF0FBECDBFDF91CF911F910F91089504
:102920000F931F93CF93DF9300D000D0CDB7DEB7C6
:102930008B01BC01CE0101960E94601462EB73E032
:10294000CE0101960E945513BC018DEC9CE00E94C3
:102950004F05CE0101960E94F912C8010E94B211E2
:1029600026960FB6F894DEBF0FBECDBFDF91CF9194
:102970001F910F910895FC0111821082138212821F
:1029800015821482FB0101900020E9F73197AF0115
:10299000461B570B0C948F13EF92FF920F931F93CC
:1029A000CF93DF931F921F92CDB7DEB78C017B01CF
:1029B00067E973E00E94BB14C7010E94C60597FD3A
:1029C0000EC08A30910559F089831A8241E050E0A7
:1029D000BE016F5F7F4FC8010E942913EDCFC80170
:1029E0000F900F90DF91CF911F910F91FF90EF907B
:1029F0000895AF92BF92CF92DF92EF92FF920F9322
:102A00001F93CF93DF93CDB7DEB72C970FB6F89413
:102A1000DEBF0FBECDBF6B017C01A42E122FB02EE6
:102A200061EC74E0CE0107960E94BB14612F70E048
:102A30008A2D90E00E94A91020E030E0A901C70192
:102A4000B6010E946C478823C1F002EB12E02B2DE7
:102A500045E0C701B6010E94FE41B801CE010196D2
:102A60000E94BB14BE016F5F7F4FCE0107960E948C
:102A7000AE12CE0101960E94F912BE01695F7F4F2E
:102A8000CE0101960E946014CE0101960E94250D90
:102A9000CE0101960E94F912CE0107960E94F9120A
:102AA0002C960FB6F894DEBF0FBECDBFDF91CF914D
:102AB0001F910F91FF90EF90DF90CF90BF90AF905C
:102AC00008950F931F93CF93DF9300D000D0CDB71D
:102AD000DEB78B01BC01CE0101960E9460146AEE44
:102AE00074E0CE0101960E945513BC018DEC9CE070
:102AF0000E944F05CE0101960E94F91269EB73E026
:102B0000012B11F066EB73E0CE0101960E94BB141D
:102B1000BE016F5F7F4F8DEC9CE00E949A12CE0148
:102B200001960E94F91226960FB6F894DEBF0FBEEA
:102B3000CDBFDF91CF911F910F9108950F931F93F8
:102B4000CF93DF9300D000D0CDB7DEB784369105A8
:102B5000F4F48C010A9774F465EC74E0CE010196EC
:102B60000E94BB14CE0101960E94250DCE01019654
:102B70000E94F912B801CE0101960E94BA13CE014B
:102B800001960E94250DCE0101960E94F91226960B
:102B90000FB6F894DEBF0FBECDBFDF91CF911F916E
:102BA0000F910895DF92EF92FF920F931F93CF93AF
:102BB000DF9300D000D0CDB7DEB77C01D62E6DEB11
:102BC00073E0CE0101960E94BB144D2D60E0CE0152
:102BD00001960E946914CE0101960E94F912F70134
:102BE00084819581969587950AE010E0081B190B62
:102BF000B701CE0101960E9460144D2D602FCE01C9
:102C000001960E946914CE0101960E94F91226963F
:102C10000FB6F894DEBF0FBECDBFDF91CF911F91ED
:102C20000F91FF90EF90DF900895FF920F931F9305
:102C3000CF93DF9300D000D0CDB7DEB7F62E142FA0
:102C4000803127E29207BCF597FF03C091958195EB
:102C500091099F938F9381ED93E09F938F9382EBE4
:102C600092E09F938F930E94554B612F70E08F2DC0
:102C700090E00E94A91062EB72E0CE0101960E94E2
:102C8000BB14CE0101960E94250DCE0101960E9433
:102C9000F9120F900F900F900F900F900F902696B3
:102CA0000FB6F894DEBF0FBECDBFDF91CF911F915D
:102CB0000F91FF900895BC01990F880B990B0E940A
:102CC000734720E030E04AE754E40E94714901E094
:102CD000212F4F2D0E94F914E2CFCF93DF9300D024
:102CE00000D0CDB7DEB765ED73E0CE0101960E944E
:102CF000BB1441E060E0CE0101960E946914CE0150
:102D000001960E94F91220E030E0A901609196023C
:102D10007091970280919802909199020E946C475D
:102D20001816C4F169ED76E0CE0101960E94BB143D
:102D300041E064E0CE0101960E946914CE01019643
:102D40000E94F91260919602709197028091980208
:102D5000909199020E94E349CB0141E066E00E9414
:102D6000151668E87DE0CE0101960E94601441E0EE
:102D70006CE0CE0101960E946914CE0101960E947A
:102D8000F91226960FB6F894DEBF0FBECDBFDF91C5
:102D9000CF91089568E87DE0CE0101960E9460140D
:102DA00041E065E0CE0101960E946914CE010196D2
:102DB0000E94F9126CED73E0CE0101960E94BB14E3
:102DC00041E06CE0CE0101960E946914CE010196AB
:102DD0000E94F91260919602709197028091980278
:102DE000909199020E94E349CB0141E06FE00E947B
:102DF0001516C7CFEF92FF920F931F93CF93DF93D8
:102E0000CDB7DEB762970FB6F894DEBF0FBECDBF69
:102E10007C018B0167E973E0CE010D960E94BB1423
:102E200060EE73E00115110529F00130110531F450
:102E300069EE73E0CE010D960E94B013B801CE0189
:102E400007960E94BA13BE01635F7F4FCE010196C1
:102E50000E946014BE01695F7F4FCE0101960E94FF
:102E60006B13BC01C7010E946014CE0101960E9441
:102E7000F912CE0107960E94F912CE010D960E941A
:102E8000F912C70162960FB6F894DEBF0FBECDBF30
:102E9000DF91CF911F910F91FF90EF900895AF9226
:102EA000BF92CF92DF92EF92FF920F931F93CF9337
:102EB000DF93CDB7DEB7A4970FB6F894DEBF0FBE91
:102EC000CDBF67E973E0CE014F960E94BB1484E446
:102ED000A82E82E0B82EF501448555856685778554
:102EE000CE0143960E94E61397E6C92E92E0D92EB2
:102EF000F6014485558566857785CE010D960E943D
:102F0000E6132AE8E22E22E0F22EF70144855585E9
:102F100066857785CE0107960E94E61364E377E025
:102F2000CE0101960E94BB14BE01695F7F4FCE01A6
:102F300001960E946B1361EF73E00E945513BE016E
:102F4000635F7F4F0E946B1361EF73E00E94551324
:102F5000BE016D5E7F4F0E946B1361EF73E00E94B4
:102F60005513BC01CE014F960E944914CE01019623
:102F70000E94F912CE0107960E94F912CE010D9619
:102F80000E94F912CE0143960E94F91208EE12E057
:102F9000F80160857185CE0149960E94BA13F80147
:102FA00066817781CE0143960E94BA1340915C08F6
:102FB00050915D0860915E0870915F08CE010D969A
:102FC0000E94E613F8014081518162817381CE0134
:102FD00001960E94E613BE016F5F7F4FCE010796F8
:102FE0000E94601461EF73E0CE0107960E945513B2
:102FF000BE01635F7F4F0E946B1361EF73E00E941D
:103000005513BE016D5E7F4F0E946B1361EF73E03D
:103010000E945513BE01675E7F4F0E946B1361EFE4
:1030200073E00E945513BC01CE014F960E94881395
:10303000CE0107960E94F912CE0101960E94F91264
:10304000CE010D960E94F912CE0143960E94F9120C
:10305000CE0149960E94F9124091E40A5091E50A86
:103060006091E60A7091E70ACE0149960E94E61344
:103070004091DA0A5091DB0A6091DC0A7091DD0A16
:10308000CE0143960E94E6134091F90A5091FA0A44
:103090006091FB0A7091FC0ACE010D960E94E61326
:1030A0004091EF0A5091F00A6091F10A7091F20A92
:1030B000CE0101960E94E613BE016F5F7F4FCE01E5
:1030C00007960E94601461EF73E0CE0107960E949C
:1030D0005513BE01635F7F4F0E946B1361EF73E076
:1030E0000E945513BE016D5E7F4F0E946B1361EF0E
:1030F00073E00E945513BE01675E7F4F0E946B1301
:1031000061EF73E00E945513BC01CE014F960E94FF
:103110008813CE0107960E94F912CE0101960E94F3
:10312000F912CE010D960E94F912CE0143960E942B
:10313000F912CE0149960E94F912F801648575854D
:1031400086859785681B790BCE010D960E94BA1370
:103150004091D00A5091D10A6091D20A7091D30A5D
:10316000CE0101960E94E613BE016F5F7F4FCE0134
:1031700007960E94601461EF73E0CE0107960E94EB
:103180005513BE01635F7F4F0E946B1361EF73E0C5
:103190000E945513BC01CE014F960E948813CE01A8
:1031A00007960E94F912CE0101960E94F912CE01F3
:1031B0000D960E94F912F60140855185628573854E
:1031C000CE0149960E94E613F6014481558166813D
:1031D0007781CE0143960E94E613F7014085518521
:1031E00062857385CE010D960E94E613F701448136
:1031F000558166817781CE0101960E94E613BE015A
:103200006F5F7F4FCE0107960E94601461EF73E0FD
:10321000CE0107960E945513BE01635F7F4F0E9447
:103220006B1361EF73E00E945513BE016D5E7F4F1B
:103230000E946B1361EF73E00E945513BE01675E3D
:103240007F4F0E946B1361EF73E00E945513BC0126
:10325000CE014F960E948813CE0107960E94F91264
:10326000CE0101960E94F912CE010D960E94F9122C
:10327000CE0143960E94F912CE0149960E94F9129E
:103280000E949E0BAB01BC01CE0143960E941C1410
:103290006091BB0A7091BC0ACE010D960E94BA13D0
:1032A000F5014085518562857385CE0101960E94A6
:1032B000E613BE016F5F7F4FCE0107960E94601438
:1032C00061EF73E0CE0107960E945513BE01635F64
:1032D0007F4F0E946B1361EF73E00E945513BE0194
:1032E0006D5E7F4F0E946B13BC01CE014F960E9412
:1032F0008813CE0107960E94F912CE0101960E9412
:10330000F912CE010D960E94F912CE0143960E9449
:10331000F912BE01615E7F4F83E99BE00E949A1221
:10332000CE014F960E94F912A4960FB6F894DEBF14
:103330000FBECDBFDF91CF911F910F91FF90EF9006
:10334000DF90CF90BF90AF900895CF92DF92EF9231
:10335000FF920F931F93CF93DF9300D000D0CDB790
:10336000DEB78C0163EF73E0CE0101960E94BB14BF
:10337000B801CE0101960E946B13BC018DEC9CE05C
:103380000E949A12CE0101960E94F91263E074E045
:10339000CE0101960E94BB1470E060E0CE01019660
:1033A0000E946115CE0101960E94F9120091190B3D
:1033B00010E06FE074E0CE0101960E94BB14B801EA
:1033C000CE0101960E946115CE0101960E94F9126C
:1033D00000917A0710E06BE174E0CE0101960E9443
:1033E000BB14B801CE0101960E946115CE01019671
:1033F0000E94F91267E274E0CE0101960E94BB14AC
:1034000070E060E0CE0101960E946115CE01019648
:103410000E94F9120091010810E063E374E0CE010C
:1034200001960E94BB14B801CE0101960E9461155D
:10343000CE0101960E94F91200915A0810E06FE344
:1034400074E0CE0101960E94BB14B801CE01019632
:103450000E946115CE0101960E94F91200910508A3
:1034600010E06BE474E0CE0101960E94BB14B80139
:10347000CE0101960E946115CE0101960E94F912BB
:103480000091790710E067E574E0CE0101960E9493
:10349000BB14B801CE0101960E946115CE010196C0
:1034A0000E94F9120091C50A10E063E674E0CE01B3
:1034B00001960E94BB14B801CE0101960E946115CD
:1034C000CE0101960E94F91200915B0810E06FE6B0
:1034D00074E0CE0101960E94BB14B801CE010196A2
:1034E0000E946115CE0101960E94F9120091C20A54
:1034F00010E06BE774E0CE0101960E94BB14B801A6
:10350000CE0101960E946115CE0101960E94F9122A
:103510000091C30A10E066E874E0CE0101960E94B3
:10352000BB14B801CE0101960E946115CE0101962F
:103530000E94F91200911D0810E060E974E0CE01CC
:1035400001960E94BB14B801CE0101960E9461153C
:10355000CE0101960E94F91208EE12E0F801E08413
:10356000F1846CE974E0CE0101960E94BB14B701AE
:10357000CE0101960E949014CE0101960E94F9128C
:10358000F801E680F78068EA74E0CE0101960E94B7
:10359000BB14B701CE0101960E949014CE01019692
:1035A0000E94F912F80160817181828193810E94E9
:1035B000E3496B0164EB74E0CE0101960E94BB14F9
:1035C000B601CE0101960E949014CE0101960E9490
:1035D000F91226960FB6F894DEBF0FBECDBFDF916D
:1035E000CF911F910F91FF90EF90DF90CF900895B2
:1035F000EF92FF920F931F93CF93DF93CDB7DEB778
:103600002C970FB6F894DEBF0FBECDBF8C017B01A7
:1036100060EC74E0CE0107960E94BB1467E973E08A
:10362000C8010E94BB14C701F7FE04C08827992770
:103630008E199F099F938F9387EC94E09F938F93AC
:1036400082EB92E09F938F930E94554B62EB72E066
:10365000CE0107960E94B0130F900F900F900F901D
:103660000F900F906CEC74E0F7FC02C06FEC73E00D
:10367000CE0101960E94BB14BE01695F7F4FCE014F
:1036800001960E946B13BC01C8010E944914CE012F
:1036900001960E94F912CE0107960E94F912C80104
:1036A0002C960FB6F894DEBF0FBECDBFDF91CF9141
:1036B0001F910F91FF90EF9008950F931F93CF9359
:1036C000DF93CDB7DEB7AA970FB6F894DEBF0FBE73
:1036D000CDBF8C0167E973E0CE0185960E94BB14D3
:1036E000F801B197EE35F10508F05DC18827E4587F
:1036F000F44E8F4F0C94324AB01FD31CD11FD41FED
:10370000D71FDD1FD31CE31FE61FE01FD31CD31CF4
:10371000D31CD31CD31CD31C851F941F971F9A1F27
:103720009D1FA01FA31FD31C821FD31CD31CD31CFF
:10373000D31CD31CA81FC51FE21CFF1E0D1FD31CCA
:10374000141F1B1F271F361F3D1F481FD31CD31CD0
:103750004F1F591FD31C5F1FD31CDA1B661FD31CBE
:10376000D31CD31C7B1FEF1FD31C2120D31CD31CC5
:10377000D31CDA1FD31CA61FD31C081F111FD31C78
:10378000431F221F2F1F391F411F4B1FD31CD31C48
:10379000561F5C1FD31C631FD31CD31C691FD31C73
:1037A000D31CD31C7F1F1E20D31CD31CE91FD31C8A
:1037B000EC1FAD1F60915C0870915D0880915E0800
:1037C00090915F0802EB12E022E044E00E94FE418B
:1037D000B801CE014F960E94BB14609150027091C7
:1037E000510280915202909153020E94E349CE010E
:1037F00049960E94F81A6091E8027091E90280915E
:10380000EA029091EB0222E044E00E94FE41B801FE
:10381000CE0143960E94BB146091730270917402B2
:1038200080917502909176020E94E349CE010D9637
:103830000E94F81A60919602709197028091980206
:10384000909199020E94E349CE0101960E94F81AD4
:10385000BE016F5F7F4FCE0107960E94601461EF3B
:1038600073E0CE0107960E945513BE01635F7F4F40
:103870000E946B1361EF73E00E945513BE016D5EF1
:103880007F4F0E946B1361EF73E00E945513BE01DE
:10389000675E7F4F0E946B1361EF73E00E945513C8
:1038A000BE01615E7F4F0E946B1361EF73E00E9467
:1038B0005513BC01CE0185960E944914CE0107968E
:1038C0000E94F912CE0101960E94F912CE010D96C6
:1038D0000E94F912CE0143960E94F912CE01499638
:1038E0000E94F912CE014F960E94F9128091D002E7
:1038F0009091D1026EEC74E0892B11F465EC74E0C8
:10390000CE0143960E94BB14809165076EEC74E073
:10391000811102C065EC74E0CE010D960E94BB14CB
:10392000809166076EEC74E0811102C065EC74E072
:10393000CE0101960E94BB14BE016F5F7F4FCE0186
:1039400007960E94601461EF73E0CE0107960E9413
:103950005513BE01635F7F4F0E946B1361EF73E0ED
:103960000E945513BE016D5E7F4F0E946B13BC0118
:10397000CE0185960E948813CE0107960E94F91207
:10398000CE0101960E94F912CE010D960E94F91205
:10399000CE0143960E94F912BE016B5D7F4F80E31A
:1039A0009CE00E949A12CE0185960E94F912AA9676
:1039B0000FB6F894DEBF0FBECDBFDF91CF911F9140
:1039C0000F9108954091500250915102609152021E
:1039D00070915302CE0143960E94E6134091730208
:1039E000509174026091750270917602CE010D962D
:1039F0000E94E613409196025091970260919802BE
:103A000070919902CE0101960E94E613BE016F5F8C
:103A10007F4FCE0107960E94601461EF73E0CE01E4
:103A200007960E945513BE01635F7F4F0E946B1380
:103A300061EF73E00E945513BE016D5E7F4F0E94DF
:103A40006B1361EF73E00E945513BC01CE018596A4
:103A50000E944914CE0107960E94F912CE010196E8
:103A60000E94F912CE010D960E94F912CE014396E2
:103A70000E94F9126091F0027091F102CE01499614
:103A80000E94BA136091EE027091EF02CE0143964C
:103A90000E94BA1340915C0850915D0860915E08E5
:103AA00070915F08CE010D960E94E6134091E802E6
:103AB0005091E9026091EA027091EB02CE01019609
:103AC0000E94E613BE016F5F7F4FCE0107960E94F2
:103AD000601461EF73E0CE0107960E945513BE019A
:103AE000635F7F4F0E946B1361EF73E00E94551379
:103AF000BE016D5E7F4F0E946B1361EF73E00E9409
:103B00005513BE01675E7F4F0E946B1361EF73E038
:103B10000E945513BC01CE0185960E948813CE01E8
:103B200007960E94F912CE0101960E94F912CE0169
:103B30000D960E94F912CE0143960E94F912CE0111
:103B400049960E94F9124091E40A5091E50A609169
:103B5000E60A7091E70ACE0149960E94E613409169
:103B6000DA0A5091DB0A6091DC0A7091DD0ACE011D
:103B700043960E94E6134091F90A5091FA0A609127
:103B8000FB0A7091FC0ACE010D960E94E61340914B
:103B9000EF0A5091F00A6091F10A7091F20ACE0199
:103BA00001960E94E613BE016F5F7F4FCE0107961C
:103BB0000E94601461EF73E0CE0107960E945513D6
:103BC000BE01635F7F4F0E946B1361EF73E00E9441
:103BD0005513BE016D5E7F4F0E946B1361EF73E062
:103BE0000E945513BE01675E7F4F0E946B1361EF09
:103BF00073E00E945513BC01CE0185960E94881384
:103C0000CE0107960E94F912CE0101960E94F91288
:103C1000CE010D960E94F912CE0143960E94F91230
:103C2000CE0149960E94F9126091F4027091F5025A
:103C30008091F6029091F702681B790BCE010D96E8
:103C40000E94BA134091D00A5091D10A6091D20AD1
:103C50007091D30ACE0101960E94E613BE016F5FF8
:103C60007F4FCE0107960E94601461EF73E0CE0192
:103C700007960E945513BE01635F7F4F0E946B132E
:103C800061EF73E00E945513BC01CE0185960E943E
:103C90008813CE0107960E94F912CE0101960E9468
:103CA000F912CE010D960E94F9126091D002709126
:103CB000D102CE0143960E94BA136091650770E06D
:103CC000CE010D960E94BA136091660770E0CE0196
:103CD00001960E94BA13BE016F5F7F4FCE01079617
:103CE0000E94601461EF73E0CE0107960E945513A5
:103CF000BE01635F7F4F0E946B1361EF73E00E9410
:103D00005513BE016D5E7F4F0E946B1361EF73E030
:103D10000E945513BC01CE0185960E948813CE01E6
:103D200007960E94F912CE0101960E94F912CE0167
:103D30000D960E94F912CE0143960E94F9120E943C
:103D40009E0BAB01BC01CE0149960E941C146091F0
:103D50001B0870911C088091390290913A02680FFB
:103D6000791FCE0143960E94BA1360911A0870E041
:103D7000CE010D960E94BA1360911D0870E0CE012D
:103D800001960E94BA13BE016F5F7F4FCE01079666
:103D90000E94601461EF73E0CE0107960E945513F4
:103DA000BE01635F7F4F0E946B1361EF73E00E945F
:103DB0005513BE016D5E7F4F0E946B1361EF73E080
:103DC0000E945513BE01675E7F4F0E946B13BC01BA
:103DD000CE0185960E948813CE0107960E94F912A3
:103DE000CE0101960E94F912CE010D960E94F912A1
:103DF000CE0143960E94F912CE014996CBCD809117
:103E0000F4029091F5029093F7028093F602CBCDE5
:103E10001092F7021092F602C6CD81E080936507FA
:103E2000C2CD10926507BFCD81E090E09093D102A2
:103E30008093D002B8CD83E090E090933A028093D3
:103E40003902B1CD10923A0210923902ACCD81E024
:103E50008093560810923B020E94310DA4CD81E060
:103E60008093560880933B0280E0F6CF109264075F
:103E70009ACD81E08093640796CD81E080936607B8
:103E800092CD109266071092D1021092D0028BCD83
:103E90001092020888CD81E08093020884CD8EE4E0
:103EA00090E09093F1028093F0027DCD89E490E060
:103EB000F8CF83E590E0F5CF88E590E0F2CF81E0A0
:103EC0008093060870CD109206086DCD0E94120DE9
:103ED0006ACD80913802882341F01092A70D60E0EE
:103EE0008BE99DE00E94630B5ECD10929A0D60E01D
:103EF0008EE89DE0F7CF81E08093010854CD1092C9
:103F0000010851CD8AE090E0CCCF8AE090E0909318
:103F1000EF028093EE029093BF028093BE029093D3
:103F20003D0280933C023FCD84E190E0F0CF8EE1F2
:103F300090E0EDCF88E290E0EACF82E390E0E7CF37
:103F40008CE390E0E4CF86E490E0E1CF10921D088E
:103F500010921C0810921B0826CD10921A08F8CF58
:103F600081E080931D0810921A0880911B0890919F
:103F70001C08181619060CF016CD9195819591091B
:103F800090931C0880931B080ECD81E080931A0843
:103F900010921D0880911B0890911C0897FF03CD7B
:103FA000ECCF82E090E0ECCF84E090E0E9CF86E0D7
:103FB00090E0E6CF88E090E0E3CF8AE090E0E0CFC9
:103FC00084E190E0DDCF88E290E0DACF8CE390E00E
:103FD000D7CF80E590E0D4CF84E690E0D1CF809138
:103FE000BE029091BF029093EF028093EE02809107
:103FF000C0029091C1029093F1028093F00210925E
:10400000D1021092D0020E94120D109265071092F8
:10401000660710923A02109239020E94A90D10927E
:104020000608109264071092020810921C08109261
:104030001B0810921A0810921D08B5CC0E94C90ED8
:10404000B2CC0E948312AFCCAF92BF92CF92DF92DC
:10405000EF92FF920F931F93CF93DF93CDB7DEB70D
:1040600062970FB6F894DEBF0FBECDBF6C017B0127
:104070005A010E942B1160ED74E0CE0101960E945E
:10408000BB1460E0CE0101960E94D215CE010196CC
:104090000E94F912B601CE0101960E94601461E0FF
:1040A000CE0101960E94D215CE0101960E94F9120E
:1040B0000E941D0E10926707F70180819181F70120
:1040C000329601E010E0219131912817390734F43C
:1040D0000F5F1F4FA016B106B4F7F1CF68EE73E083
:1040E00080E090E00E940F050E946C0E8091C30A50
:1040F00081112FC08091C20A882311F00F5F1F4FDA
:10410000A016B10614F401E010E06DED74E0CE01EC
:1041100001960E94BB1462E0CE0101960E94D21566
:10412000CE0101960E94F912F801EE0FFF1FEE0D6D
:10413000FF1D60817181CE0101960E94FA1663E035
:10414000CE0101960E94D215CE0101960E94F9126D
:10415000C5CF0E942B116DED74E0CE0101960E9437
:10416000BB1460E0CE0101960E94D215CE010196EB
:104170000E94F912B601CE0101960E94601461E01E
:10418000CE0101960E94D215CE0101960E94F9122D
:10419000000F111F0E0D1F1DF80160817181CE01EE
:1041A00007960E94FA1667EE74E0CE0101960E940F
:1041B000BB14BE01695F7F4FCE0101960E946B1355
:1041C000BC01CE010D960E94601462E0CE010D96F6
:1041D0000E94D215CE010D960E94F912CE010196D1
:1041E0000E94F912CE0107960E94F91268EE73E060
:1041F00080E090E00E940F05F80180819181629635
:104200000FB6F894DEBF0FBECDBFDF91CF911F91E7
:104210000F91FF90EF90DF90CF90BF90AF900895F7
:104220000F931F93CF93DF93CDB7DEB72C970FB6C5
:10423000F894DEBF0FBECDBF1A86198621E030E0AC
:104240003C872B8718861F82BC01CE0101960E94F5
:10425000601442E050E0BE01695F7F4FCE010196DD
:104260000E9424208C01CE0101960E94F912C801FF
:104270002C960FB6F894DEBF0FBECDBFDF91CF9165
:104280001F910F91089585ED8093BC0080916B0B79
:1042900090916C0BA0916D0BB0916E0B0796A11DC8
:1042A000B11D23E0B695A795979587952A95D1F7E7
:1042B0002091BC0024FD03C01092690B0895409129
:1042C0006B0B50916C0B60916D0B70916E0B452BCD
:1042D000462B472B69F30097A105B10541F02AE26F
:1042E0002A95F1F700C00197A109B109E1CF8091AA
:1042F0006A0B0C94D309CF92DF92EF92FF920F9347
:104300001F93CF93DF9300D000D0CDB7DEB76EEC14
:1043100076E083E99BE00E943D1209EE13E083E919
:104320009BE00E94FE05892BE9F461E070E080E0EB
:1043300090E00E940F050150110989F7C12CD12C82
:104340007601C701B60126960FB6F894DEBF0FBE00
:10435000CDBFDF91CF911F910F91FF90EF90DF9034
:10436000CF90089583E99BE00E94FE05892B31F3ED
:1043700063E97BE0CE0101960E94CC1489819A8189
:10438000C12CD12C7601009721F00E9441436B0192
:104390007C01CE0101960E94F912D3CF8F929F9299
:1043A000AF92BF92CF92DF92EF92FF9280915A0824
:1043B00090915B089111D3C08111C9C00E940D0971
:1043C0001092E80A10921E08C090E802D090E9020C
:1043D000E090EA02F090EB026091EE027091EF0241
:1043E000072E000C880B990B0E9473474B015C0150
:1043F000AC019B01C701B6010E946C4787FFAAC0B0
:1044000020E030E0A901C701B6010E94194A181640
:104410000CF0A0C081E08093E80AA7019601C501D5
:10442000B4010E94044920E030E04AE754E40E94CD
:10443000D24720E030E04AE754E40E9405490E9458
:10444000EA49683E83E0780710F468EE73E0693B60
:104450008BE0780710F068EB7BE070930C086093BA
:104460000B086091F2027091F302072E000C880B8A
:10447000990B0E9473474B015C01AC019B01C70182
:10448000B6010E94194A87FD06C01092F7021092E9
:10449000F60210921F0880911F08882379F1A50168
:1044A0009401C701B6010E946C4787FF27C081E0D5
:1044B0008093E80AA7019601C501B4010E9404494E
:1044C00020E030E04AE754E40E94D24720E030E0A8
:1044D0004AE754E40E9405490E94EA49683E83E0A5
:1044E000780710F468EE73E0693B8BE0780710F012
:1044F00068EB7BE070930C0860930B086091F0020E
:104500007091F102072E000C880B990B0E947347E3
:104510009B01AC01C701B6010E94194A18160CF0A4
:104520004FC01092E80A81E080931E0810920C0898
:1045300010920B0870E060E089E0FF90EF90DF9050
:10454000CF90BF90AF909F908F900C94F0030E94FB
:104550007B2136CF10920C0810920B0882CF81116C
:1045600038C060E08BE39BE00E9413100E94870834
:104570006093E8027093E9028093EA029093EB0261
:104580000E940D09C090E802D090E902E090EA0292
:10459000F090EB0220E030E042EB52E4C701B601BC
:1045A0000E946C4787FD0AC020E030E040E251ECF9
:1045B000C701B6010E94194A181614F410925B083C
:1045C000FF90EF90DF90CF90BF90AF909F908F9033
:1045D00008950E947B21D6CF4F925F927F928F9257
:1045E0009F92AF92BF92CF92DF92EF92FF920F9382
:1045F0001F93CF93DF93CDB7DEB7C457D1090FB662
:10460000F894DEBF0FBECDBF8DEC9CE00E94CC02C3
:104610001092B8071092B7071092700B1092920B7D
:104620000E94B5098BED9AE09093DB078093DA073F
:104630008CED9AE09093DF078093DE0781E0809312
:104640006F0B8FE38093910B0E94F409811102C0DC
:104650001092380261E08DE30E94B4038DE390E094
:1046600090937D0780937C071092B00D809100009D
:104670008E010F5F1F4F803109F46DC0B80190E0CB
:1046800080E00E941508882309F465C08D818F336E
:1046900009F461C08FE38D838091B50D9091B60DC3
:1046A0000E94DD0770E060E08091B50D9091B60D3D
:1046B0000E94BE0740E06EE48091B50D9091B60D6A
:1046C0000E948A0740E06B818091B50D9091B60DF4
:1046D0000E948A0740E06C818091B50D9091B60DE3
:1046E0000E948A0780910000803141F040E06D8196
:1046F0008091B50D9091B60D0E948A078091B50DFD
:104700009091B60D2091B20D222319F10E94DD0780
:10471000882309F140E06CEC8091B50D9091B60DC5
:104720000E948A074091AC0D68E48091B50D90918C
:10473000B60D0E948A078091AC0D81112EC064E1F4
:1047400070E080E090E00E940F058091B50D90919F
:10475000B60D0E94DD078AE08093AF0D8091B30D06
:104760008230B0F1F12C8091B30DF81688F580916C
:10477000AF0D8C3069F16F2DC8010E941310898133
:10478000803121F1C8010E94E3089091AF0D981784
:1047900010F48093AF0DF394E6CF8091AD0D882394
:1047A00029F060E08091AE0D0E94860364E170E024
:1047B00080E090E00E940F058091AD0D882329F2E2
:1047C00061E08091AE0D0E948603BFCF8CE0DDCF0B
:1047D00080913802882309F475C08BE99DE00E941E
:1047E000CE10E091B50DF091B60D138615861486A6
:1047F0001286118610861782168215821482138201
:104800001092B30D1092B40DFF24F394B80180916F
:10481000B50D9091B60D0E94930F882309F45EC0E8
:1048200067E0C8010E94200798858913EFCF809127
:10483000B30D8F5F8093B30D8981883231F008F01A
:1048400044C0803111F0823209F78091B40D8F5F3E
:104850008093B40D8091AC0D811126C08091B50D6F
:104860009091B60D0E94DD07B8018091B50D909131
:10487000B60D0E94BE0740E064EB8091B50D9091AB
:10488000B60D0E948A078091B50D9091B60D0E94D9
:104890003707E82E8091B50D9091B60D0E94DD0787
:1048A000E11002C0F092AC0D89818031A9F0C801FD
:1048B0000E94E3089091AF0D981708F0A7CF80935E
:1048C000AF0DA4CF8EE89DE08ACF8B3309F4BDCF26
:1048D000823409F09BCFB9CF8CE0ECCF0E94120D4F
:1048E0000E948C116091E4027091E5028091E602D1
:1048F0009091E7029B01AC010E946C4781110E94DC
:1049000051128091E4029091E502A091E602B091EB
:10491000E70280933E0290933F02A0934002B0933F
:1049200041028093BE0A9093BF0AA093C00AB0933D
:10493000C10A81E08093B10261E089E00E94B40382
:1049400061E08AE00E94B40361E08EE30E94B40358
:1049500061E08FE30E94B40361E080E40E94B4034D
:1049600061E083E40E94B40362E087E00E94B40344
:1049700062E086E00E94B40362E085E00E94B40336
:1049800062E084E00E94B40362E083E00E94B4032A
:1049900062E082E00E94B40362E08DE00E94B40312
:1049A00062E08CE00E94B40362E08BE00E94B403FA
:1049B00062E085E40E94B40362E084E40E94B403F0
:1049C00062E082E40E94B40362E083E40E94B403E4
:1049D00062E081E40E94B40362E082E40E94B403D6
:1049E0000E942B111092C40A109273070E946C0E41
:1049F0008091BD0A811110C28091C20A882309F4F6
:104A000059C06EEE74E0C8010E94BB1460E0C8019A
:104A10000E94D215C8010E94F9126DEF74E0C8011E
:104A20000E94BB1461E0C8010E94D215C8010E9417
:104A3000F9126CE075E0C8010E94BB1462E0C80185
:104A40000E94D215C8010E94F9126DE175E0C801FB
:104A50000E94BB1443E060E0C8010E946914C801D1
:104A60000E94F91265E0E62EF12CDD24D394E114C6
:104A7000F10401F10E941D0E0E946C0E80916707E7
:104A80008823A9F310926707B701C8010E94BA13DF
:104A900043E062E1C8010E946914C8010E94F91252
:104AA00081E0E81AF1088091BD0A882301F3D092D1
:104AB0007307DDCF8091C30A882309F467C066E2DB
:104AC00075E0C8010E94BB1460E0C8010E94D215C5
:104AD000C8010E94F9126DEF74E0C8010E94BB1476
:104AE00061E0C8010E94D215C8010E94F9126CE071
:104AF00075E0C8010E94BB1462E0C8010E94D21593
:104B0000C8010E94F9126DE175E0C8010E94BB1452
:104B100043E060E0C8010E946914C8010E94F912D4
:104B200055E0E52EF12CDD24D394E114F10471F16C
:104B30000E941D0E0E946C0E809167078823A9F3C6
:104B400010926707B701C8010E94BA1343E062E1FF
:104B5000C8010E946914C8010E94F912E1E0EE1A2E
:104B6000F1088091BD0A882301F3D092C40A0E9403
:104B70002B1166E275E0C8010E94BB1460E0C80119
:104B80000E94D215C8010E94F912CFCF80917307FD
:104B9000882309F441C10E942B1163E375E0C80129
:104BA0000E94BB1460E0C8010E94D215C8010E9497
:104BB000F91260ED77E080E090E00E940F050E941E
:104BC0008C1163E475E0C8010E94BB1462E575E0D6
:104BD000CE0107960E94BB1461E675E0CE010D96EA
:104BE0000E94BB1462E775E0CE0143960E94BB149D
:104BF00060E875E0CE0149960E94BB1462E975E059
:104C0000CE014F960E94BB1462EA75E0CE018596F4
:104C10000E94BB1461EB75E0CE018B960E94BB1421
:104C20006DEB75E0CE01C1960E94BB147E01F7E5E5
:104C3000EF0EF11CF70116861786108A118A8091F3
:104C4000BE029091BF02918380838091C0029091B7
:104C5000C102938382838091CA029091CB02958393
:104C600084838091CC029091CD029783868380913A
:104C7000CE029091CF02918780878091D00290914F
:104C8000D102938782878091E2029091E302958717
:104C90008487D12CC12C57010E942B110E946C0ECD
:104CA0008091C20A882329F0FFEFCF1ADF0A0E9401
:104CB0002B1189E0C816D10414F0D12CC12C86E048
:104CC0008C9D40018D9D900C1124800E911EB4018D
:104CD000CE01C7960E94601460E0CE01C7960E9484
:104CE000D215CE01C7960E94F912F601EE0FFF1FF2
:104CF000EA0DFB1D60817181CE01C7960E94FA16F4
:104D000062E0CE01C7960E94D215CE01C7960E94DE
:104D1000F91268EE73E080E090E00E940F050E94B7
:104D20006C0E7090C30A772009F4B6CFF601319764
:104D3000E830F10570F48827EF55F94D8F4F0C944A
:104D4000324AC32A122B672BBC2B0B2C602CE92C6C
:104D5000002D4090BE025090BF02B401CE01815997
:104D60009F4F0E9460148AE090E09AAF89AF84E17F
:104D700090E09CAF8BAF8EE190E09EAF8DAF88E26C
:104D800090E021969FAF8EAF219782E390E023962B
:104D90009FAF8EAF239758AE4FAABE0161597F4F88
:104DA000CE0187599F4F0E94601445E050E0BE013C
:104DB000695C7F4FCE0187599F4F0E9424204C0190
:104DC000CE0187599F4F0E94F9129092BF028092A4
:104DD000BE02CE0181599F4F0E94F9128091BE02FE
:104DE0009091BF02F5019183808368EE73E080E0CB
:104DF00090E00E940F0571104FCF7E01E7E3EE0EA9
:104E0000F11CF6E0EF1AF108C7010E94F9120E1525
:104E10001F05B9F7109273070E942B116EEC75E015
:104E2000CE01895A9F4F0E94BB1462ED75E0C80104
:104E30000E94BB14BE01695A7F4FC8010E946B13C8
:104E4000BC01CE01C7960E946014C8010E94F912ED
:104E5000BE01695C7F4FC8010E94601460E0C80118
:104E60000E94D215C8010E94F9126CED75E0C801CC
:104E70000E94BB1462E0C8010E94D215C8010E94C2
:104E8000F91268EE75E0C8010E94BB1463E0C80126
:104E90000E94D215C8010E94F91268EE73E080E00A
:104EA00090E00E940F050E942B11CE01C7960E9430
:104EB000F912CE01895A9F4F0E94F912FFB6F89459
:104EC00080917407811127C0E6EDF4E08491ECE154
:104ED000F5E09491E82FF0E0EE0FFF1FE35FFB4F4A
:104EE000A591B491EC91E92321F461E085E30E945E
:104EF000860361E085E30E94B4038CB580618CBDBC
:104F00008CB580648CBD61E084E30E94B40361E0F1
:104F100083E30E94B403809174078F5F80937407CA
:104F2000FFBE80917A00887F80937A0080917A001A
:104F3000856080937A0080917E00816080937E00FE
:104F400080917E00826080937E0080917E008460EC
:104F500080937E0080917E00806180937E008091AE
:104F60007E00806280937E0060E089E00E9486037C
:104F700061E08EE30E94860361E08FE30E94860376
:104F800061E080E40E94860370E060E089E00E94B6
:104F9000F00360E08BE39BE00E9413100E940D0978
:104FA0008091380240E352E060E0882309F441C573
:104FB0008BE99DE00E943C1148E252E061E08BE900
:104FC0009DE00E943C1140E252E062E08BE99DE0EE
:104FD0000E943C1148E152E063E08BE99DE00E94B1
:104FE0003C1140E152E064E08BE99DE00E943C11FD
:104FF00048E052E065E08BE99DE00E943C1140E012
:1050000052E066E08BE99DE00E943C111092190B82
:1050100061E081E10E94B40360E081E10E948603C7
:1050200068EE73E080E090E00E940F0560E081E1AF
:105030000E94B40381E10E945D03FF24F394009772
:1050400009F4F12CF0927B07892B19F081E0809311
:10505000190B69EF75E0C8010E94BB146F2D70E059
:10506000C8010E946115C8010E94F91280E39CE00A
:105070000E94CC021092180B60E076E08DEC9CE070
:105080000E94A8118FE00E945D030E94B21161E0AE
:105090008FE00E94B40360E08FE00E94860368EE18
:1050A00073E080E090E00E940F0560E08FE00E94D6
:1050B000B4038FE00E945D03FF24F394892B09F46D
:1050C000F12CF092180B6BE076E0C8010E94BB1443
:1050D0006F2D70E0C8010E946115C8010E94F9128D
:1050E000E090180BEE2021F083E99BE00E94CC02B7
:1050F00087E00E945D036C0181E0C114D10409F0D6
:1051000080E080937A0786E00E945D0321E00097AB
:1051100009F020E020930108EE2039F0892B29F4D2
:1051200081E080935A081092010885E00E945D0397
:105130005C0181E0A114B10409F080E080930508CE
:1051400084E00E945D034C0181E08114910409F028
:1051500080E08093790783E00E945D03FF24F3944D
:10516000892B09F0F12CF092780782E00E945D0310
:1051700077247394892B09F0712C709277078DE056
:105180000E945D03892B19F581E08093C50A88EEA2
:1051900093E090937607809375078CE00E945D03FF
:1051A000892B31F48CED95E0909376078093750709
:1051B0008BE00E945D03892B51F4809175079091DB
:1051C000760788519C4F909376078093750761E02E
:1051D0008AE00E94B40361E088E00E94B40370E0BA
:1051E00060E08AE00E94F00370E060E088E00E94E6
:1051F000F0031092C30A1092C20A0E946C0E892812
:1052000051F48EE490E09093F1028093F002909339
:10521000C1028093C002872D90E0880F991F8F0DE7
:10522000911D8230910509F434C48330910509F44D
:1052300033C4019709F42AC488E290E090933D02B8
:1052400080933C0280913C0290913D029093EF024A
:105250008093EE029093BF028093BE02C114D104EA
:1052600009F01DC483E090E090933A0280933902E4
:10527000F0907B07FF2019F081E08093190B0E94CA
:105280002B116EEC75E0CE0181599F4F0E94BB142B
:1052900062ED75E0C8010E94BB14BE0161597F4FE9
:1052A000C8010E946B13BC01CE0187599F4F0E9419
:1052B0006014C8010E94F912CD2839F462E176E049
:1052C000CE0187599F4F0E947E13AB2839F46BE1C2
:1052D00075E0CE0187599F4F0E947E13809101088F
:1052E000882339F064E176E0CE0187599F4F0E9410
:1052F0007E13FF2039F06AE077E0CE0187599F4F97
:105300000E947E13EE2039F062E177E0CE018759EA
:105310009F4F0E947E1380915A08882339F06EECCB
:1053200076E0CE0187599F4F0E947E138091C50A77
:10533000882339F066E176E0CE0187599F4F0E94BD
:105340007E13BE0167597F4FCE0101960E94601403
:10535000CE0101960E94A519CE0101960E94F91274
:1053600080910508882341F061E08AE00E94B4033F
:1053700060E08AE00E948603BE0167597F4FCE013C
:1053800001960E94601460E0CE0101960E94D21541
:10539000CE0101960E94F91280917A07882379F054
:1053A00068E176E0CE0101960E94BB1461E0CE0177
:1053B00001960E94D215CE0101960E94F9128091A9
:1053C0000508882379F06AE276E0CE0101960E9412
:1053D000BB1462E0CE0101960E94D215CE01019667
:1053E0000E94F9126091F0027091F102CE010196D3
:1053F0000E94BA136091EE027091EF02CE01C7963F
:105400000E94BA136DE376E0CE01895A9F4F0E9445
:10541000BB14BE01695C7F4FCE01895A9F4F0E9429
:105420006B1364E476E00E945513BE016F5F7F4FFB
:105430000E946B136DE476E00E945513BC01CE010F
:1054400087599F4F0E944914CE01895A9F4F0E944D
:10545000F912CE01C7960E94F912CE0101960E9460
:10546000F912BE0167597F4FCE0101960E94601468
:1054700062E0CE0101960E94D215CE0101960E94F3
:10548000F9126FE476E0CE0101960E94BB1443E06E
:1054900060E0CE0101960E946914CE0101960E943F
:1054A000F91260913E0270913F028091400290910A
:1054B000410204E023E04CE00E94F91480911D08B1
:1054C000882309F4F1C260EC72E1CE01C7960E9414
:1054D000BA136DE576E0CE01895A9F4F0E94BB1446
:1054E000BE01695C7F4FCE01895A9F4F0E946B13AA
:1054F00064E176E00E945513BC01CE0101960E9442
:10550000601463E0CE0101960E94D215CE0101968F
:105510000E94F912CE01895A9F4F0E94F912CE01C2
:10552000C7960E94F91280E690E090931C08809341
:105530001B0868E873E180E090E00E940F05CE014F
:1055400087599F4F0E94F912CE0181599F4F0E94A7
:10555000F9121092D1021092D0020E942B116BE628
:1055600076E0CE0101960E94BB1461E0CE01019667
:105570000E94D215CE0101960E94F912F12CE12C65
:1055800010E000E098C28090C0029090C102BE017D
:10559000695F7F4FCE0181599F4F0E94601484E460
:1055A00090E09AAF89AF89E490E09CAF8BAF8EE436
:1055B00090E09EAF8DAF83E590E021969FAF8EAFD8
:1055C000219788E590E023969FAF8EAF239798AE02
:1055D0008FAABE0161597F4FCE0187599F4F0E940C
:1055E000601445E050E0BE01695C7F4FCE018759F1
:1055F0009F4F0E9424204C01CE0187599F4F0E944B
:10560000F9129092C1028092C002CE0181599F4F3F
:105610000E94F9128091C0029091C102F701938318
:105620008283E3CB8090CA029090CB02BE01635F7D
:105630007F4FCE0181599F4F0E94601480ED97E00B
:105640009AAF89AF84EC99E09CAF8BAF88EB9BE07D
:105650009EAF8DAF8CEA9DE021969FAF8EAF2197D4
:1056600080EA9FE023969FAF8EAF239784E991E174
:1056700025969FAF8EAF259798AE8FAABE01615930
:105680007F4FCE0187599F4F0E94601446E050E043
:10569000BE01695C7F4FCE0187599F4F0E94242035
:1056A0004C01CE0187599F4F0E94F9129092CB0274
:1056B0008092CA02CE0181599F4F0E94F9128091B7
:1056C000CA029091CB02F701958384838ECB8090A0
:1056D000CC029090CD02BE016D5E7F4FCE0181590C
:1056E0009F4F0E94601484EB90E09AAF89AF8AEFDD
:1056F00090E09CAF8BAF8CE291E09EAF8DAF8EE5DA
:1057000091E021969FAF8EAF219780E991E023969B
:105710009FAF8EAF239782EC91E025969FAF8EAF1F
:10572000259798AE8FAABE0161597F4FCE01875948
:105730009F4F0E94601446E050E0BE01695C7F4FBD
:10574000CE0187599F4F0E9424204C01CE018759DA
:105750009F4F0E94F9129092CD028092CC02CE010E
:1057600081599F4F0E94F9128091CC029091CD02F5
:10577000F7019783868339CB8090CE029090CF0239
:10578000BE01675E7F4FCE0181599F4F0E9460141A
:1057900084EF91E09AAF89AF88EE93E09CAF8BAF36
:1057A0008CED95E09EAF8DAF80ED97E021969FAF99
:1057B0008EAF219784EC99E023969FAF8EAF23970D
:1057C00098AE8FAABE0161597F4FCE0187599F4F76
:1057D0000E94601445E050E0BE01695C7F4FCE013D
:1057E00087599F4F0E9424204C01CE0187599F4F1B
:1057F0000E94F9129092CF028092CE02CE0181597E
:105800009F4F0E94F9128091CE029091CF02F70132
:1058100091878087EACA8090D0029090D102BE0121
:10582000615E7F4FCE0181599F4F0E94601484EFCB
:1058300091E09AAF89AF88EE93E09CAF8BAF80ED9B
:1058400097E09EAF8DAF88EB9BE021969FAF8EAF28
:10585000219780EA9FE023969FAF8EAF239788E839
:1058600093E125969FAF8EAF259798AE8FAABE0184
:1058700061597F4FCE0187599F4F0E94601446E0C7
:1058800050E0BE01695C7F4FCE0187599F4F0E9457
:1058900024204C01CE0187599F4F0E94F91290920B
:1058A000D1028092D002CE0181599F4F0E94F912FD
:1058B0008091D0029091D102F7019387828795CA97
:1058C0008090E2029090E302BE016B5D7F4FCE01BB
:1058D00081599F4F0E9460141AAE19AE85E090E086
:1058E0009CAF8BAF8AE090E09EAF8DAF8FE090E0F1
:1058F00021969FAF8EAF219784E190E023969FAFD2
:105900008EAF239789E190E025969FAF8EAF2597C4
:105910008EE190E027969FAF8EAF279783E290E0CD
:1059200029969FAF8EAF299788E290E02B969FAF84
:105930008EAF2B978DE290E02D969FAF8EAF2D9777
:1059400082E390E02F969FAF8EAF2F9787E390E092
:1059500061969FAF8EAF61978CE390E063969FAFA7
:105960008EAF639781E490E065969FAF8EAF6597A9
:1059700084E690E067969FAF8EAF679798AE8FAA48
:10598000BE0161597F4FCE0187599F4F0E9460141D
:105990004FE050E0BE01695C7F4FCE0187599F4FB9
:1059A0000E9424204C01CE0187599F4F0E94F9127A
:1059B0009092E3028092E202CE0181599F4F0E94B1
:1059C000F9128091E2029091E302F70195878487B2
:1059D0000CCABE01655D7F4FCE01C7960E94601460
:1059E000CE01C7960E9410214C01CE01C7960E949D
:1059F000F9128A94892811F40E946B11712CF5C94F
:105A0000BE016F5C7F4FCE01C7960E946014CE012D
:105A1000C7960E9410214C01CE01C7960E94F91230
:105A20008A94892809F0E1C90E9451120E948312C8
:105A3000DCC98EE89DE00E943C1148E252E061E042
:105A40008EE89DE00E943C1140E252E062E08EE868
:105A50009DE00E943C1148E152E063E08EE89DE049
:105A60000E943C1140E152E064E08EE89DE00E941B
:105A70003C1148E052E065E08EE89DE00E943C1158
:105A800040E052E066E08EE89DE0BECA8EE190E024
:105A9000D5CB84E190E0D2CB8AE090E0CFCB1092DE
:105AA0003A0210923902E4CB10921C0810921B08A3
:105AB00040CDF12CE12C8090E8029090E902A0907A
:105AC000EA02B090EB0220E030E042EB52E4C50184
:105AD000B4010E94194A181654F020E030E040E862
:105AE0005FE3C501B4010E946C4787FF88C08091C5
:105AF0005A08811103C160E08BE39BE00E94131000
:105B00000E9487086093E8027093E9028093EA029A
:105B10009093EB0264EF71E080E090E00E940F054B
:105B20000E940D098FEFE81AF80AE3E0EE16F1047F
:105B30000CF4C1CF64E275E0CE0101960E94BB1463
:105B400042E0602FCE0101960E946914CE010196B9
:105B50000E94F9120F5F1F4F043111050CF4A9CFF9
:105B60006BE776E0CE0101960E94BB14CE01019650
:105B70000E94A519CE0101960E94F9120E942B11D4
:105B800069E876E0CE0101960E94BB1461E0CE0187
:105B900001960E94D215CE0101960E94F9126BE97E
:105BA00076E0CE0101960E94BB1462E0CE01019620
:105BB0000E94D215CE0101960E94F91260ED77E0A5
:105BC00080E090E00E940F0520E030E04EEF52ECC4
:105BD0006091E8027091E9028091EA029091EB02F3
:105BE0000E946C478111CACC1092E8021092E9021F
:105BF0001092EA021092EB0281E080935B080E940F
:105C00002B1120E030E048EC52E46091E802709102
:105C1000E9028091EA029091EB020E94D2470E9431
:105C2000E3499B01685E734069357B4110F020EACF
:105C30003FE0E0E6F8E088EB9AE0219331938E179D
:105C40009F07D9F78091EE029091EF029093C902DD
:105C50008093C8020E94CE218091C50A81110E94C2
:105C6000A40E20913E0230913F024091400250919B
:105C7000410260E070E080E89FE30E947149609318
:105C8000010B7093020B8093030B9093040B0E9403
:105C90000D090E9487086B017C0120E030E040E2A2
:105CA00051EC0E946C4787FD54C0C092E802D0922C
:105CB000E902E092EA02F092EB020E944205609350
:105CC000100B7093110B8093120B9093130BCC5805
:105CD000DF4F0FB6F894DEBF0FBECDBFDF91CF917F
:105CE0001F910F91FF90EF90DF90CF90BF90AF90FA
:105CF0009F908F907F905F904F9008950E947B219E
:105D00006093E8027093E9028093EA029093EB02B9
:105D100068EE73E080E090E00E940F056801FFEFFD
:105D2000CF1ADF0A69EA76E0CE0101960E94BB1421
:105D300042E0602FCE0101960E946914CE010196C7
:105D40000E94F91286E0C816D1040CF055CF8601E6
:105D5000B2CE1092E8021092E9021092EA0210927A
:105D6000EB02ABCF1F920F920FB60F9211242F931D
:105D70003F938F939F93AF93BF938091330B9091F9
:105D8000340BA091350BB091360B3091320B23E0E0
:105D9000230F2D3758F50196A11DB11D2093320B0D
:105DA0008093330B9093340BA093350BB093360B49
:105DB0008091370B9091380BA091390BB0913A0B31
:105DC0000196A11DB11D8093370B9093380BA093C2
:105DD000390BB0933A0BBF91AF919F918F913F9147
:105DE0002F910F900FBE0F901F90189526E8230F4C
:105DF0000296A11DB11DD2CF1F920F920FB60F9226
:105E000011240BB60F922F933F934F935F936F9391
:105E10007F938F939F93AF93BF93EF93FF9383E908
:105E20009BE00E942806FF91EF91BF91AF919F9157
:105E30008F917F916F915F914F913F912F910F9033
:105E40000BBE0F900FBE0F901F9018951F920F92D0
:105E50000FB60F9211240BB60F922F933F934F93CF
:105E60005F936F937F938F939F93AF93BF93EF93C2
:105E7000FF9383E99BE00E948A05FF91EF91BF9118
:105E8000AF919F918F917F916F915F914F913F91D2
:105E90002F910F900BBE0F900FBE0F901F90189573
:105EA0001F920F920FB60F9211240BB60F922F93E1
:105EB0003F934F935F936F937F938F939F93AF9392
:105EC000BF93EF93FF9380E39CE00E942806FF912D
:105ED000EF91BF91AF919F918F917F916F915F9162
:105EE0004F913F912F910F900BBE0F900FBE0F90CF
:105EF0001F9018951F920F920FB60F9211240BB698
:105F00000F922F933F934F935F936F937F938F9352
:105F10009F93AF93BF93EF93FF9380E39CE00E9426
:105F20008A05FF91EF91BF91AF919F918F917F91E2
:105F30006F915F914F913F912F910F900BBE0F90FA
:105F40000FBE0F901F9018951F920F920FB60F92D1
:105F500011240BB60F922F933F934F935F936F9340
:105F60007F938F939F93AF93BF93EF93FF938DECAA
:105F70009CE00E942806FF91EF91BF91AF919F9105
:105F80008F917F916F915F914F913F912F910F90E2
:105F90000BBE0F900FBE0F901F9018951F920F927F
:105FA0000FB60F9211240BB60F922F933F934F937E
:105FB0005F936F937F938F939F93AF93BF93EF9371
:105FC000FF938DEC9CE00E948A05FF91EF91BF91B9
:105FD000AF919F918F917F916F915F914F913F9181
:105FE0002F910F900BBE0F900FBE0F901F90189522
:105FF0001F920F920FB60F9211240BB60F922F9390
:106000003F934F935F936F937F938F939F93AF9340
:10601000BF93EF93FF938091B900887F803609F496
:106020004DC008F040C0883209F4A9C028F580317D
:1060300009F49DC0C8F4882309F4FBC0883009F432
:1060400096C0FF91EF91BF91AF919F918F917F91FA
:106050006F915F914F913F912F910F900BBE0F90D9
:106060000FBE0F901F901895883109F488C08032B8
:1060700041F78093670B14C0803409F49DC040F44D
:106080008033B9F38833E9F68093670B85ECB0C0B1
:10609000803509F485C0883509F496C0883489F6BE
:1060A0000E944321CECF883909F48CC038F5883757
:1060B00029F050F4883611F0803719F683E0809388
:1060C000690B1092000857C0883809F47BC08039EA
:1060D00019F0803809F0B5CF80910008803208F0BF
:1060E00071C0E091000881E08E0F809300088091DC
:1060F000BB00F0E0E052F84F80833DC0803B39F0B8
:10610000E0F4803A09F479C0883A09F09ACF84E043
:106110008093690B1092DD071092DC07E091DA079B
:10612000F091DB0719958091DC0781110FC081E0A8
:106130008093DC071092BA0709C0803C09F4A6CF0F
:10614000883C09F4A3CF883B09F07BCFE091DD07C1
:1061500081E08E0F8093DD07F0E0E654F84F8081F8
:106160008093BB009091DD078091DC0729C080916E
:10617000440B8093BB0085EC8093BC0062CF909170
:10618000660B8091650B981758F5E091660B81E0DE
:106190008E0F8093660BF0E0EB5BF44F8081E9CFCC
:1061A000E091660B81E08E0F8093660B8091BB00BF
:1061B000F0E0EB5BF44F80839091660B8091650B70
:1061C0009817C8F285E8D8CFE091660B81E08E0F72
:1061D0008093660B8091BB00F0E0EB5BF44F808313
:1061E0008091680B81115CCF81E08093430B84EA3E
:1061F0008093BC001092690B24CF85EC8093BC0087
:106200001092690B80910008803230F4E091000810
:10621000F0E0E052F84F10826091000870E0E091E9
:10622000DE07F091DF0780EE97E0199510920008E5
:1062300008CF1092670B34CFCF93DF9300D000D0FC
:10624000CDB7DEB7E3E9FBE01382128288EE93E07C
:10625000A0E0B0E084839583A683B78327E433E08E
:106260003183208345E351E05587448744E351E07F
:106270005787468740E351E0518B408B41E351E023
:10628000538B428B42E351E0558B448B46E351E004
:10629000578B468B118E128E138E148EE0E3FCE02A
:1062A0001382128284839583A683B78331832083EC
:1062B00045ED50E05587448744ED50E057874687C9
:1062C00040ED50E0518B408B41ED50E0538B428BC1
:1062D00042ED50E0558B448B46ED50E0578B468B9A
:1062E000118E128E138E148EEDECFCE0138212824E
:1062F00084839583A683B7833183208325EC30E0A4
:106300003587248724EC30E03787268720EC30E07F
:10631000318B208B21EC30E0338B228B22EC30E070
:10632000358B248B26EC30E0378B268B118E128E2A
:10633000138E148EEAE6FDE0138212828483958325
:10634000A683B78389E593E09183808360E089E346
:106350000E94B403E0E2F5E0E491A3ECBDE0EC932D
:10636000EAEDF4E0E491F0E0EE0FFF1FE957FB4F98
:106370008591949112969C938E9311971B961C92E3
:106380001B971D961C921D971C961C921C971A9683
:106390001C921A9719961C92199718961C92189786
:1063A00017961C92179716961C92169715961C9284
:1063B000159714961C92149713961C921397ECEA57
:1063C000FDE0168A158A1182B287A187178210868E
:1063D000108289E0838381E084838583868388EECD
:1063E00093E09093AB0D8093AA0D80EF9AE0909389
:1063F000A90D8093A80DEBE9FDE0138212822BE634
:1064000033E031832083118687E2848394E192878D
:1064100084E083871486EEE8FDE0138212823183E4
:10642000208311862FE3248392878387148668EC68
:1064300073E088E89DE00E94BB146EEC75E082E892
:106440009DE00E94BB146BEA76E0CE0101960E94AB
:10645000BB1462E87DE0CE0101960E946B13BC0183
:106460008CE79DE00E946014CE0101960E94F91213
:1064700067E973E086E79DE00E94BB140E94420535
:1064800026960FB6F894DEBF0FBECDBFDF91CF9139
:106490000895CF93DF93CDB7DEB7A6970FB6F894E4
:1064A000DEBF0FBECDBF789484B5826084BD84B555
:1064B000816084BD85B5826085BD85B5816085BDFF
:1064C00080916E00816080936E00109281008091B7
:1064D000810082608093810080918100816080933F
:1064E0008100809180008160809380008091B10064
:1064F00084608093B1008091B00081608093B0008F
:1065000080919100826080939100809191008160E0
:1065100080939100809190008160809390008091A1
:10652000A10082608093A1008091A100816080938E
:10653000A1008091A00081608093A0008091210142
:1065400082608093210180912101816080932101EB
:106550008091200181608093200180917A00846085
:1065600080937A0080917A00826080937A00809193
:106570007A00816080937A0080917A0080688093AD
:106580007A001092C1000E94EC221E012CE0220E23
:10659000311C80902E0B90902F0BA090300BB09060
:1065A000310B80922A0B90922B0BA0922C0BB09265
:1065B0002D0B4090260B5090270B6090280B70906D
:1065C000290B4092220B5092230B6092240B709265
:1065D000250B8AE390E00E94F50C6B017C01C092D0
:1065E0002E0BD0922F0BE092300BF092310BAC01BE
:1065F0009B01C301B2010E940549A50194010E94BB
:10660000044924EA30E74DE75FE30E94D2472B01BB
:106610003C014092260B5092270B6092280B7092FF
:10662000290B8090AD029090AE02A090AF02B09086
:10663000B002A5019401C701B6010E9404496B0193
:106640007C01C0921E0BD0921F0BE092200BF092A7
:10665000210B10911D0B10931C0B01E020E030E08A
:10666000A901C301B2010E94194A18160CF000E0FA
:1066700000931D0B8BE390E00E94F50C60938A025F
:1066800070938B0280938C0290938D02A5019401EC
:106690000E940449A70196010E94D2479B01AC01C8
:1066A0006091A6027091A7028091A8029091A90220
:1066B0000E9405496093A6027093A7028093A802E6
:1066C0009093A90287E390E00E94F50C6093670223
:1066D000709368028093690290936A02A501940105
:1066E0000E940449A70196010E94D2479B01AC0178
:1066F000609183027091840280918502909186025C
:106700000E940549609383027093840280938502FE
:106710009093860288E390E00E94F50C6093440217
:10672000709345028093460290934702A50194011D
:106730000E940449A70196010E94D2479B01AC0127
:106740006091600270916102809162029091630297
:106750000E94054960936002709361028093620217
:106760009093630280911A0B90911B0B019690936A
:106770001B0B80931A0B20E030E0A901C301B2018A
:106780000E94194A18160CF02FC2113009F42CC2BD
:106790008091190B882309F492C080E39CE00E9449
:1067A000FE05181619060CF08AC080E39CE00E94D2
:1067B000B2057C0184E5E816F10409F05DC060E3F0
:1067C0007CE0CE0181960E94CC14BE016F5D7F4FAC
:1067D000CE014B960E9460146EEC76E0CE010196DD
:1067E0000E94BB14BE01655E7F4FCE0101960E94E0
:1067F0006B13BC01CE0145960E946014CE01019638
:106800000E94F912098D1A8D0115110509F040C079
:106810001982FE01319620E030E0A901119180ED4E
:10682000810F8A3098F4AAE0B0E00E94C848212F76
:10683000110F330B205331098901330F220B330B16
:10684000A9019801260F371F481F591F2E163F0612
:1068500029F7CA01B9010E94790B81E08093090BE5
:10686000CE0145960E94F912CE014B960E94F91274
:10687000CE0181960E94F91280E39CE00E94FE0501
:1068800018161906CCF480E39CE00E94B205F4CF00
:106890000331110510F003E110E06D897E89A80134
:1068A000CE0101960E94464BE1E0F0E0EC0FFD1FA7
:1068B000E00FF11F1082ADCFC7010E945D1B8091D8
:1068C000180B8823A1F183E99BE00E94FE051816AE
:1068D00019066CF583E99BE00E94B20583349105AB
:1068E000B1F463E97BE0CE0101960E94CC14CE01A5
:1068F00001960E94F91283E99BE00E94FE0518169A
:106900001906ACF483E99BE00E94B205F4CF84340D
:10691000910519F40E944F17EECF8035910559F774
:1069200083E99BE00E94B2050E945D1BE4CF0E94B8
:1069300042056093100B7093110B8093120B909390
:10694000130B603DA7E07A078105910560F468515B
:106950007C4F8F4F9F4F60930C0B70930D0B809368
:106960000E0B90930F0B8091C80A9091C90A019663
:106970009093C90A8093C80A2AE037ED43E25CE3AA
:106980006091140B7091150B8091160B9091170B61
:106990000E94D2479B01AC016091AD027091AE02A2
:1069A0008091AF029091B0020E9405496093AD02C0
:1069B0007093AE028093AF029093B0028090A602D3
:1069C0009090A702A090A802B090A90240903E0229
:1069D00050903F026090400270904102E0901A0B8C
:1069E000F0901B0B0091C60A1091C70AA5019401F3
:1069F00060919A0270919B0280919C0290919D02FD
:106A00000E94054960939A0270939B0280939C02B6
:106A100090939D02209183023091840240918502DF
:106A2000509186026091770270917802809179028C
:106A300090917A020E9405496093770270937802E0
:106A40008093790290937A022091600230916102E2
:106A5000409162025091630260915402709155021C
:106A600080915602909157020E940549609354020A
:106A700070935502809356029093570280911108AB
:106A80008111D0C580910D0890910E08A0910F083A
:106A9000B09110080196A11DB11D80930D0890932F
:106AA0000E08A0930F08B09310088D329140A105F5
:106AB000B1051CF081E08093110880911E088823A5
:106AC00009F429C670E060E089E00E94F0031092AA
:106AD000BC0A1092BB0A1092070810920808109284
:106AE000090810920A0810920C0810920B08809165
:106AF0000508882309F446C00091AA0D1091AB0D3A
:106B000020E030E04CE552E46091E8027091E90247
:106B10008091EA029091EB020E94194A87FD07C01A
:106B20008091A80D9091A90D801791072CF000314C
:106B3000AEE01A0709F0F0C68091D0029091D10220
:106B400030E020E0892B59F42FEF30E0D8010E948B
:106B50003A4A20E13EE040E050E00E94A9483093EC
:106B600004082093030880910608882321F01092DE
:106B700004081092030860910308709104088AE0E9
:106B80000E94F0031092A6021092A7021092A8028F
:106B90001092A90210928302109284021092850230
:106BA00010928602109260021092610210926202AC
:106BB000109263028091050B9091060B20911A0BA5
:106BC00030911B0B820F931F9093060B8093050B44
:106BD00010921B0B10921A0B1092140B1092150BA3
:106BE0001092160B1092170B4091100B5091110B35
:106BF0006091120B7091130B80910C0B90910D0B07
:106C0000A0910E0BB0910F0B481759076A077B072D
:106C100008F4EAC40E94420568517C4F8F4F9F4F91
:106C200060930C0B70930D0B80930E0B90930F0BD6
:106C30006091050B7091060B072E000C880B990BC9
:106C40000E9473472091010B3091020B4091030B7E
:106C50005091040B0E94D2476B017C01C092FD0A47
:106C6000D092FE0AE092FF0AF092000BAC019B0169
:106C700060919A0270919B0280919C0290919D027A
:106C80000E9471494B015C0180929602909297029A
:106C9000A0929802B092990220E030E0A9010E94EF
:106CA000194A18160CF03DC66091F70A7091F80A5F
:106CB000072E000C880B990B0E947347A5019401C5
:106CC0000E9405490E94E3497093F80A6093F70A0D
:106CD00020E030E040E85FE36091F30A7091F40A4D
:106CE0008091F50A9091F60A0E9405496093F30A93
:106CF0007093F40A8093F50A9093F60A20E030E04E
:106D000041E655E4C501B4010E9471499B01AC0103
:106D100060919202709193028091940290919502F9
:106D20000E940549609392027093930280939402AB
:106D300090939502A7019601609177027091780275
:106D40008091790290917A020E9471494B015C0115
:106D500020E030E0A9010E946C4787FD29C680929F
:106D6000730290927402A0927502B092760220E0B3
:106D700030E040EF51E460917302709174028091B1
:106D80007502909176020E946C4787FF08C01092AE
:106D90007302109274021092750210927602809023
:106DA000730290907402A0907502B09076021091D8
:106DB000E80A20E030E048E453E4C501B4010E9451
:106DC000194A18169CF4111111C08091180890915D
:106DD000190801968C33910509F4EFC590931908B1
:106DE000809318081092080B1092070B20E030E0F7
:106DF00041E655E4C501B4010E9471492B013C01F3
:106E0000112309F4F9C56091E20A7091E30A072E93
:106E1000000C880B990B0E947347A50194010E94F6
:106E200005490E94E3497093E30A6093E20A20E077
:106E300030E040E85FE36091DE0A7091DF0A809104
:106E4000E00A9091E10A0E9405496093DE0A70937E
:106E5000DF0A8093E00A9093E10AA3019201609116
:106E60006B0270916C0280916D0290916E020E9493
:106E7000054960936B0270936C0280936D0290934E
:106E80006E02A701960160915402709155028091A3
:106E90005602909157020E9471496B017C0120E0DB
:106EA00030E0A9010E946C4787FDE5C5C092500201
:106EB000D0925102E0925202F092530220E030E070
:106EC00040E752E460915002709151028091520269
:106ED000909153020E946C4787FF08C010925002A5
:106EE000109251021092520210925302C09050021E
:106EF000D0905102E0905202F09053026091CE0A7D
:106F00007091CF0A072E000C880B990B0E947347D3
:106F1000A70196010E9405490E94E3497093CF0A98
:106F20006093CE0A20E030E040E85FE36091CA0A57
:106F30007091CB0A8091CC0A9091CD0A0E940549AC
:106F40006093CA0A7093CB0A8093CC0A9093CD0ABF
:106F500020E030E041E655E4C701B6010E947149E6
:106F60009B01AC0160914C0270914D0280914E02E8
:106F700090914F020E94054960934C0270934D021C
:106F800080934E0290934F021092060B1092050BC5
:106F900010929A0210929B0210929C0210929D02F3
:106FA00010927702109278021092790210927A026F
:106FB00010925402109255021092560210925702EB
:106FC0008091C80A9091C90A9093C70A8093C60A13
:106FD0001092C90A1092C80A8091C50A882309F440
:106FE00081C00E94DD0C65E070E00E941E4A892B82
:106FF00009F078C0609173027091740280917502FB
:10700000909176022091E80A211190580E94E3495C
:10701000072E000C880B990B0E9473472091960253
:107020003091970240919802509199020E9405492F
:107030000E94E34977FF02C070E060E0809112088F
:10704000909113080196893191050CF019C5909320
:10705000130880931208E0911208F0911308EE0FC4
:10706000FF1FE05EF74F7183608302E218E022E5C4
:10707000C22E28E0D22E7801812C912C5401F701E8
:10708000619171917F0190E080E00E9471479B01C6
:10709000AC01C501B4010E9405494B015C01CE144D
:1070A000DF0469F720E030E040EC51E40E947149D0
:1070B0000E94EA49709353086093520820913B0262
:1070C000222309F4E0C4683C710560F480E00E946A
:1070D000310D84E598E0D8011D921D928D018A172B
:1070E0009B07C9F78091C40A81110C945B41809180
:1070F000090B70E060E0882309F4CDC48FE090E0D4
:107100000E94A9100E94ED0C0E949E1560ED76E091
:10711000CE0101960E94BB14CE0101960E94250D5E
:10712000CE0101960E94F9120E94E50C0E949E1564
:107130002091BB0A3091BC0A032E000C440B550B66
:107140002951310941095109A4E6B0E00E94C8481B
:1071500026EE30E040E050E00E94A948122F67E997
:1071600073E0CE014B960E94BB1464ED76E0CE0135
:107170004B960E94B0138091AA0D9091AB0D803177
:107180009E4039F46CED76E0CE014B960E94B01330
:1071900015E68091E80A882309F46AC0C090E802E5
:1071A000D090E902E090EA02F090EB028091C30AED
:1071B0008823B1F06091EE027091EF02072E000C6F
:1071C000880B990B0E947347A70196010E94194AE8
:1071D000181634F464EE76E0CE014B960E94B0139C
:1071E00060913C0270913D02072E000C880B990BB8
:1071F0000E947347A70196010E94194A181634F499
:107200006CEE76E0CE014B960E94B01380911F0881
:10721000882361F08091C20A60EC76E0882311F047
:1072200068EC76E0CE014B960E94B01320E030E08F
:1072300048E453E460917302709174028091750286
:10724000909176020E946C4787FF42C464EF76E01B
:10725000CE0101960E94BB14BE016F5F7F4FCE012D
:107260004B960E94AE12CE0101960E94F91215E6CD
:1072700080911E08882339F06CEF76E0CE014B96A2
:107280000E94B01315E680915B08882339F064E012
:1072900077E0CE014B960E94B01315E680911D0851
:1072A000882341F16CE077E0CE014B960E94B01349
:1072B00060911B0870911C08CE0145960E94BA137C
:1072C000BE016B5E7F4FCE0101960E9460146DEC93
:1072D00073E0CE0101960E945513BC01CE014B967E
:1072E0000E948813CE0101960E94F912CE014596A4
:1072F0000E94F91280911A08882341F160E177E039
:10730000CE014B960E94B01360911B0870911C082F
:10731000CE0145960E94BA13BE016B5E7F4FCE012F
:1073200001960E9460146DEC73E0CE0101960E94FC
:107330005513BC01CE014B960E948813CE010196D5
:107340000E94F912CE0145960E94F91280915408CC
:10735000882339F064E177E0CE014B960E94B013A8
:1073600015E68FEF810F843608F4BAC3BE01655E5F
:107370007F4FCE0101960E94601440E067E0CE018D
:1073800001960E946914CE0101960E94F912CE0165
:107390004B960E94F9120E946D168091BA0A8230B3
:1073A00009F4FEC508F0DEC3813009F478C4809189
:1073B000BA0A853008F07DC78F5F8093BA0AC09003
:1073C000CA0AD090CB0AE090CC0AF090CD0A20E017
:1073D00030E040E850E4C701B6010E94194A18168F
:1073E0000CF0C7C06091ED0A7091EE0A072E000CF8
:1073F000880B990B0E9473472091E90A3091EA0AA1
:107400004091EB0A5091EC0A0E9471496093EF0A97
:107410007093F00A8093F10A9093F20A1092E90AAD
:107420001092EA0A1092EB0A1092EC0A1092EE0AFD
:107430001092ED0A6091F70A7091F80A072E000C7D
:10744000880B990B0E9473472091F30A3091F40A3C
:107450004091F50A5091F60A0E9471496093F90A29
:107460007093FA0A8093FB0A9093FC0A1092F30A35
:107470001092F40A1092F50A1092F60A1092F80A85
:107480001092F70A6091D80A7091D90A072E000C61
:10749000880B990B0E9473472091D40A3091D50A2A
:1074A0004091D60A5091D70A0E9471496093DA0A36
:1074B0007093DB0A8093DC0A9093DD0A1092D40A61
:1074C0001092D50A1092D60A1092D70A1092D90AB1
:1074D0001092D80A6091E20A7091E30A072E000C1C
:1074E000880B990B0E9473472091DE0A3091DF0AC6
:1074F0004091E00A5091E10A0E9471496093E40AC8
:107500007093E50A8093E60A9093E70A1092DE0AE8
:107510001092DF0A1092E00A1092E10A1092E30A38
:107520001092E20A6091CE0A7091CF0A072E000CE9
:10753000880B990B0E947347A70196010E9471491D
:107540006093D00A7093D10A8093D20A9093D30AA1
:107550008091180B81110E944F171092CA0A109245
:10756000CB0A1092CC0A1092CD0A1092CF0A109238
:10757000CE0A0E94E50C20910A0B30910B0B82176A
:10758000930731F00E94E50C90930B0B80930A0B4C
:107590000E94ED0C20914202309143028217930722
:1075A00019F10E94ED0C9093430280934202809166
:1075B000F6029091F70201969093F7028093F602FB
:1075C0008091070B9091080B01969093080B809384
:1075D000070B2091090B222309F4FCC60E94ED0C35
:1075E000892B11F40E94C90E20911E0B30911F0BA4
:1075F0004091200B5091210B6091140B7091150B51
:107600008091160B9091170B0E9405496093140B03
:107610007093150B8093160B9093170B0E94B7066F
:107620000C94C932A3019201C501B4010E94D24752
:107630004B015C01B701FF0C880B990B0E9473474B
:107640009B01AC01C501B4010E9471496B017C0131
:10765000B801110F880B990B0E9473479B01AC0175
:10766000C701B6010E9471496B017C01609139022A
:1076700070913A02072E000C880B990B0E947347F9
:107680009B01AC01C701B6010E9404496B017C015A
:107690006091AA0D7091AB0D072E000C880B990B11
:1076A0000E9473479B01AC01C701B6010E940549C6
:1076B0000E94E3497093AB0D6093AA0D20911D08C1
:1076C000211104C020911A08222359F020911B088F
:1076D00030911C08C901860F971F9093AB0D8093C2
:1076E000AA0D8091AA0D9091AB0D81319E4034F08E
:1076F00080E19EE09093AB0D8093AA0D8091AA0D3E
:107700009091AB0D97FFD9C988EE93E09093AB0DA4
:107710008093AA0DD2C98091E80A811124C01092E9
:107720000C0810920B08A091AA0DB091AB0DA93EC8
:1077300093E0B9070CF4DFC08091D0029091D102A0
:1077400030E020E0892B51F42FEF30E00E943A4ADC
:1077500020E13EE040E050E00E94A9483093BC0A9E
:107760002093BB0A84C080910108811190C0A4E9D4
:10777000B1E1B0930C08A0930B0804E911E18091EA
:1077800002086FEF70E081116EC020E030E0A901C7
:1077900060910708709108088091090890910A0883
:1077A0000E946C4781110CC080E090E0A0E0BFE334
:1077B0008093070890930808A0930908B0930A08DB
:1077C000B801110F880B990B0E9473472091730227
:1077D0003091740240917502509176020E940449E2
:1077E00020E030E84BE355E40E9471492AE037ED90
:1077F00043E25CE30E94D2472091070830910808D9
:107800004091090850910A080E9405496B017C01CA
:1078100020E030E040E85FE30E94194A18160CF4BB
:107820005DC0C0920708D0920808E0920908F09263
:107830000A0820E030E04FE753E4609107087091B8
:1078400008088091090890910A080E94D2470E9476
:10785000E3496F3F710519F014F06FEF70E077FFA7
:1078600002C070E060E07093BC0A6093BB0A809134
:107870000608882321F01092BC0A1092BB0A60917E
:10788000BB0A7091BC0A89E00E94F00330C92091C4
:10789000960230919702409198025091990260E0CF
:1078A00070EC88EA95EC0E9404499B01AC01609160
:1078B00073027091740280917502909176020E9419
:1078C00004490E94E3498B0177FD29CF70930C088E
:1078D00060930B08672B09F052CF25CF80E090E032
:1078E000A0E8BFE38093070890930808A0930908D5
:1078F000B0930A089ECF1092BC0A1092BB0A109255
:107900000708109208081092090810920A081092AD
:107910000C0810920B08ABCF1092040810920308C9
:1079200022C96091ED0A7091EE0A072E000C880BB7
:10793000990B0E947347A50194010E9404490E947B
:10794000E3497093EE0A6093ED0A20E030E040E8EE
:107950005FE36091E90A7091EA0A8091EB0A9091E5
:10796000EC0A0E9405496093E90A7093EA0A809341
:10797000EB0A9093EC0A20E030E041E655E4C501C3
:10798000B4010E9471499B01AC0160918E0270911B
:107990008F0280919002909191020E94054960931C
:1079A0008E0270938F028093900290939102C2C9CD
:1079B000B7FAB094B7F8B094D2C9109219081092DF
:1079C0001808809116089091170801968C3391053C
:1079D00029F0909317088093160804CA109217088C
:1079E00010921608809114089091150801969093B2
:1079F000150880931408F6C96091D80A7091D90AC5
:107A0000072E000C880B990B0E947347A501940167
:107A10000E9405490E94E3497093D90A6093D80AED
:107A200020E030E040E85FE36091D40A7091D50A2D
:107A30008091D60A9091D70A0E9405496093D40A92
:107A40007093D50A8093D60A9093D70AA301920126
:107A500060916F0270917002809171029091720238
:107A60000E94054960936F027093700280937102C7
:107A70009093720206CAF7FAF094F7F8F09416CAD7
:107A800081E090E0E4CA693E734008F42BCB81E0CA
:107A90000E94310D27CB8FE090E00E94A9108091C9
:107AA0001408909115080E949E1562ED76E0CE01B3
:107AB00001960E94BB14CE0101960E94250DCE01B5
:107AC00001960E94F91280911608909117082ECB0A
:107AD000BE01655E7F4FCE0101960E946014BCCB53
:107AE00070E060E087E090E00E94A9101E5F212F07
:107AF00030E0ACE0B0E00E94F54824E630E040E041
:107B000050E00E94A948122F00E0011110C011237B
:107B100049F081E090E00E945F1111500F5F073043
:107B2000A1F735CC90E080E00E945F11F7CF0630DE
:107B300039F485E090E01123B9F386E090E0F4CFCA
:107B4000123030F084E090E00E945F111250E6CFD6
:107B500083E090E0113011F082E090E00E945F112C
:107B600010E0DCCF833009F4B9C2843009F01FCCB7
:107B70008091B80A9091B90A8C32914024F0109209
:107B8000B90A1092B80AE090B80AF090B90A8701D1
:107B9000000F111F005A174FD8016D917C91072ECD
:107BA000000C880B990B0E94734720E030E048ECF2
:107BB00052E40E9471492B013C018090E8029090B0
:107BC000E902A090EA02B090EB02BFEFEB1AFB0AC9
:107BD000F092B90AE092B80A20E030E048EC52E4B2
:107BE000C501B4010E94D2470E94E349F8017183A4
:107BF0006083A3019201C501B4010E9404496B0195
:107C00007C01C0925C08D0925D08E0925E08F09220
:107C10005F0880915B088111CACB8091C20A8111F3
:107C2000C6CB8091C30A8111C2CB20E030E0A9010C
:107C3000C701B6010E946C4787FF32C320E030E0E5
:107C400048E453E4609150027091510280915202D5
:107C5000909153020E946C4787FFA9CB6091BE02AE
:107C60007091BF02072E000C880B990B0E9473477E
:107C70002B013C01AC019B01C501B4010E946C4782
:107C800087FF95CBA7019601C301B2010E94044969
:107C90000E94E3497093EF026093EE0288CB20E0EC
:107CA00030E040E85FE3609173027091740280916C
:107CB0007502909176020E94194A18160CF0FDC0C8
:107CC0008091E80A8823C1F16CE177E0CE0101964A
:107CD0000E94BB1442E060E0CE0101960E9469144C
:107CE000CE0101960E94F9126091730270917402A4
:107CF00080917502909176020E94E349CB0142E0A7
:107D000066E00E94151663E277E0CE0101960E94BC
:107D1000BB1442E06CE0CE0101960E946914CE01D2
:107D200001960E94F91260916B0270916C02809131
:107D30006D0290916E023BC068E277E0CE01019641
:107D40000E94BB1442E060E0CE0101960E946914DB
:107D5000CE0101960E94F912609173027091740233
:107D600080917502909176020E94E349CB0142E036
:107D700066E00E9415168091560881111FC063E2CB
:107D800077E0CE0101960E94BB1442E06CE0CE0188
:107D900001960E946914CE0101960E94F912609129
:107DA0006F027091700280917102909172020E9434
:107DB000E349CB0142E06FE00E941516809156081E
:107DC000882309F4F4CA80913B0266EB76E08111C6
:107DD00002C06BEB76E0CE0101960E94BB1442E03C
:107DE0006CE0CE0101960E946914CE0101960E94BA
:107DF000F912009152081091530862EC74E0CE0120
:107E00004B960E94BB1462E070E08FE090E00E940D
:107E1000A9100115110571F1C80117FF04C08827C9
:107E20009927801B910B9F938F938BE397E09F93F0
:107E30008F9382EB92E09F938F930E94554B62EB5E
:107E400072E0CE0101960E94BB14BE016F5F7F4FAE
:107E5000CE014B960E94AE12CE0101960E94F912FD
:107E60000F900F900F900F900F900F906CEC74E0AC
:107E700017FD02C06FEC73E0CE0101960E94BB14A7
:107E8000BE01655E7F4FCE0101960E946B13BC015F
:107E9000CE0145960E946014CE0145960E94250DA4
:107EA000CE0145960E94F912CE0101960E94F91268
:107EB000CE014B960E94F9127ACA20E030E040E8E9
:107EC0005FE360916F0270917002809171029091F6
:107ED00072020E94194A181694F56FE277E0CE01FB
:107EE00001960E94BB1442E060E0CE0101960E9420
:107EF0006914CE0101960E94F91260916F0270918F
:107F0000700280917102909172020E94E349CB014C
:107F100042E066E00E94151620E030E040E85FE3B2
:107F200060916B0270916C0280916D0290916E0273
:107F30000E94194A18161CF566E377E0E6CE68E859
:107F40007DE0CE0145960E9460146CEC73E0CE019A
:107F500045960E945513BC01CE0101960E94601403
:107F600042E060E0CE0101960E946914CE010196C4
:107F70000E94F912CE0145960E94F912CDCF68E811
:107F80007DE0CE0101960E94601442E06CE0CE01DB
:107F900001960E946914CE0101960E94F9120ECF3B
:107FA00020E030E040E85FE36091500270915102C0
:107FB00080915202909153020E94194A18160CF0B7
:107FC0003FC060E477E0CE0101960E94BB1443E01D
:107FD00060E0CE0101960E946914CE0101960E94D4
:107FE000F912609150027091510280915202909169
:107FF00053020E94E349CB0143E066E00E9415165C
:1080000063E277E0CE0101960E94BB1443E06CE08E
:10801000CE0101960E946914CE0101960E94F912C8
:1080200060914C0270914D0280914E0290914F02EE
:108030000E94E349CB0143E06FE00E941516B7C9E7
:1080400020E030E040E85FE360914C0270914D0227
:1080500080914E0290914F020E94194A1816F4F432
:1080600067E477E0CE0101960E94BB1443E060E034
:10807000CE0101960E946914CE0101960E94F91268
:1080800060914C0270914D0280914E0290914F028E
:108090000E94E349CB0143E066E0CFCF68E87DE092
:1080A000CE0101960E9460146CEC73E0CE01019643
:1080B0000E945513BC01CE0145960E94601443E016
:1080C00060E0CE0145960E946914CE0145960E945B
:1080D000F912CE0101960E94F91269C98091F80245
:1080E0008111D9C080915A08882309F49AC00E944E
:1080F0007B216B017C0120E030E0A9010E94194A3C
:1081000018160CF091C0C092E802D092E902E092F9
:10811000EA02F092EB02109259081092580810925D
:108120005B080E946C0E8091570881118091C50AEE
:108130008093560880915508882321F08091C50AC4
:10814000811182C01092540880915B08811192C005
:1081500080913C0290913D029093EF028093EE0259
:108160009093BF028093BE026091E8027091E90291
:108170008091EA029091EB0202E020E040E00E9450
:10818000F9141A8219821C821B821E821D828FEDB5
:108190008D8B1E8ABE016B5E7F4FCE0101960E94C1
:1081A000B01340E065E0CE0101960E946914CE0153
:1081B00001960E94F9128091C20A882381F06EE430
:1081C00077E0CE0101960E94BB1440E065E0CE014D
:1081D00001960E946914CE0101960E94F9128091C5
:1081E000C30A8823D1F060E577E0CE0101960E94B2
:1081F000BB1440E065E0CE0101960E946914CE01F7
:1082000001960E94F91282E390E09093EF0280932E
:10821000EE029093BF028093BE0281E08093F80249
:10822000C6C80E94870865CF809158089091590868
:108230000196909359088093580821E00B970CF40D
:1082400020E020935B086DCF81E0809354080E946A
:10825000A40E8091520890915308892B09F474CF91
:10826000E2E2F8E084E598E0119211928E179F0700
:10827000D9F76ACF62E577E0CE0101960E94BB1480
:1082800040E060E0CE0101960E946914CE010196A3
:108290000E94F912C2CF1092F8020E94CE2168CC3F
:1082A0008091BE029091BF029093EF028093EE0204
:1082B0007EC881E082C80E946C0E0E946D1680917B
:1082C000C30A8823B1F027E137EB41ED58E3609111
:1082D0003E0270913F0280914002909141020E94C3
:1082E000054960933E0270933F0280934002909351
:1082F00041028091C20A8823B1F027E137EB41EDBA
:1083000058E360913E0270913F028091400290914B
:1083100041020E94044960933E0270933F028093A1
:1083200040029093410269E577E0CE0101960E94F8
:10833000BB1442E060E0CE0101960E946914CE01B8
:1083400001960E94F91260913E0270913F02809165
:1083500040029091410204E022E046E00E94F914BC
:108360006091BE0A7091BF0A8091C00A9091C10AC3
:1083700022E04EE00E94F9148091BD0A811112C0E2
:1083800080913E0290913F02A0914002B091410243
:108390008093E4029093E502A093E602B093E70293
:1083A0000E946B1120913E0230913F0240914002A9
:1083B0005091410260E070E080E89FE30E947149C3
:1083C0006093010B7093020B8093030B9093040B4B
:1083D0000C94DF3909970CF407C904C986E79DE0BE
:1083E0000E94F9128CE79DE00E94F91282E89DE05C
:1083F0000E94F91288E89DE00C94F912EF920F9315
:108400001F93CF93DF93E80134E047FD34E1042E5E
:10841000000C550B57FF03C0519541955109E32EB0
:10842000022F242FAE010E948C43CE01DF91CF9109
:108430001F910F91EF9008950F931F93CF93DF93A8
:108440008230910510F482E090E0E091D30DF0913C
:10845000D40D30E020E0B0E0A0E0309799F4211591
:10846000310509F44AC0281B390B24303105D8F5F1
:108470008A819B816115710589F1FB019383828358
:10848000FE0111C0408151810281138148175907B3
:10849000E0F04817590799F4109761F012960C9381
:1084A000129713961C933296CF01DF91CF911F91B3
:1084B0000F9108950093D30D1093D40DF4CF21158F
:1084C000310551F04217530738F0A901DB019A0139
:1084D000BD01DF01F801C1CFEF01F9CF9093D40DB9
:1084E0008093D30DCDCFFE01E20FF31F81939193C3
:1084F0002250310939832883D7CF2091D10D309173
:10850000D20D232B41F42091FB023091FC023093D9
:10851000D20D2093D10D2091F9023091FA0221154C
:10852000310541F42DB73EB74091FD025091FE0256
:10853000241B350BE091D10DF091D20DE217F3071A
:10854000A0F42E1B3F0B2817390778F0AC014E5FC3
:108550005F4F2417350748F04E0F5F1F5093D20D21
:108560004093D10D819391939FCFF0E0E0E09CCFB9
:10857000CF93DF930097E9F0FC01329713821282C8
:10858000A091D30DB091D40DED0130E020E0109713
:10859000A1F420813181820F931F2091D10D309160
:1085A000D20D2817390709F061C0F093D20DE0937E
:1085B000D10DDF91CF910895EA01CE17DF07E8F5DD
:1085C0004A815B819E0141155105B1F7E901FB83A9
:1085D000EA8349915991C40FD51FEC17FD0761F447
:1085E000808191810296840F951FE9019983888388
:1085F000828193819B838A83F0E0E0E012968D91E3
:108600009C9113970097B9F52D913C911197CD014D
:108610000296820F931F2091D10D3091D20D281711
:10862000390739F6309751F51092D40D1092D30DC9
:10863000B093D20DA093D10DBCCFD383C283408120
:108640005181840F951FC817D90761F44E5F5F4FA2
:1086500088819981480F591F518340838A819B816A
:10866000938382832115310509F0B0CFF093D40DA7
:10867000E093D30D9ECFFD01DC01C0CF13821282A7
:10868000D7CF662777270C940545BB274A3031F4AE
:10869000992322F4BDE2909581959F4F0C947343EA
:1086A000BB27FA01A62F6217710581059105330BCF
:1086B00030FB66F0AA27660F771F881F991FAA1F35
:1086C000A21710F0A21B63953850A9F7A05DAA333A
:1086D00008F0A95DA19336F7B111B1931082CA01D8
:1086E0000C945C47BB27FB015527AA27880F991FCD
:1086F000AA1FA41710F0A41B83955051B9F7A05DD1
:10870000AA3308F0A95DA193009779F7B111B1934D
:108710001192CB010C945C478F929F92AF92BF92C3
:10872000CF92DF92EF92FF920F931F93CF93DF933D
:1087300000D000D000D0CDB7DEB76A01F22EB02E47
:10874000102FFBE3AF2EA01608F41BE31F5F012FD1
:1087500027E0AE014F5F5F4F0E946346BC018981F5
:10876000982F9970913009F44EC09BE2E1FC04C04F
:108770009E2D9170E0FC49C05E2D5071E82FE8708D
:1087800083FF55C084E0911101C083E0EF2DE81B09
:108790008F1508F0E0E0D6018E2F20E25523C9F1B5
:1087A000992329F0D6019C93C60101966C0196018C
:1087B0002D5F3F4FE2FE33C08EE4D6018C9391E4EF
:1087C00011969C93119712968C93D9018E2F90E25B
:1087D00081112AC0E20FF32FF11D10828EEF9FEF5F
:1087E00029960FB6F894DEBF0FBECDBFDF91CF91B3
:1087F0001F910F91FF90EF90DF90CF90BF90AF90BF
:108800009F908F9008959DE2B7CF90E2B5CF2D93C2
:1088100081508111FCCFCE0ED11CE0E0C1CF8EE69D
:10882000D6018C9391E6CCCF9D938150D1CF482F28
:10883000447082FF3DC084E0911101C083E08F1538
:1088400010F4EF2DE81BD6018E2F20E2552309F1FD
:10885000992329F0D6019C93C60101966C019601DB
:108860002D5F3F4FE2FE1BC089E4D6018C938EE45E
:1088700011968C93119786E412968C93D9018E2FC2
:1088800090E2882309F4A6CF9D938150FACF2D93CF
:1088900081508111FCCFCE0ED11CE0E0D9CF89E60A
:1088A000D6018C938EE611968C93119786E6E4CFD1
:1088B0009B0177FF02C030E020E0A1E0B0E0911121
:1088C00002C0B0E0A0E0F9013196AE0FBF1F8B2CC3
:1088D000912CBB2009F461C05401EFEFAE1ABE0A1F
:1088E000AA0DBB1DFA161B0619F014F04F2D4A1BDA
:1088F000511188C0E3FC59C07601A42FB0E2A11148
:108900004FC0C40ED11C992309F45BC040E0D601CE
:108910001196F60190836D01552309F448C0012F8B
:10892000060F9A81582F507184FF03C0913309F4C8
:10893000015010160CF047C0093008F008E0EEE2D4
:10894000FE2E5B01A01AB1088501919481949108D3
:108950002F3F320729F4D601FC92F60131966F01C0
:108960006217730794F1021713077CF5DB01A21B52
:10897000B30BAA24A394B12CAC0EBD1EAA0DBB1D33
:1089800011968C9121503109D6011196281539057F
:10899000F4F0F60180836D01DBCFB12CA12CA0CFC8
:1089A000F701B1937F01A150AACF9111B0CFD601A9
:1089B000942F50E302C05D9391509111FCCFC40EEF
:1089C000D11C40E0ACCF01E0BACF80E3DBCF62172F
:1089D000730731F4963388F4953311F4552369F015
:1089E000F6018083FD01842F90E2811108C0A40F5D
:1089F000B11D1C9290E080E0F3CE81E3F1CF919322
:108A00008150F3CF911183CF8ACF8F929F92AF92F3
:108A1000BF92CF92DF92EF92FF920F931F93CF936B
:108A2000DF935C017B016115710519F0DB018D930A
:108A30009C9385010F5F1F4FF501D0818D2F90E032
:108A40000E943B476C01892BB9F5DD32B9F50F5F08
:108A50001F4FD5011196DC91C1E05801F1E0AF1A2A
:108A6000B10843E050E060EC72E0C5010E94444769
:108A7000892B69F5680182E0C80ED11C45E050E001
:108A80006BEB72E0C6010E944447892B21F4680118
:108A900097E0C90ED11CE114F10419F0D701CD9271
:108AA000DC9260E070E080E89FEFC111FFC060E001
:108AB00070E080E89FE7FAC05801BBCFDB3229F4B1
:108AC00085010E5F1F4FF501D181C0E0C6CF43E0A5
:108AD00050E068EB72E0C5010E944447892BE9F041
:108AE000F80110E000E020E030E0A9015F01B0ED06
:108AF0008B2E8D0E89E08815C8F19C2E689491F814
:108B00008C2F8870C2FF16C0811102C00F5F1F4FEB
:108B10003196D501DC91C92DE9CFE114F10429F09A
:108B20000E5F1F4FF7011183008360E070E080EC5F
:108B30009FE7BCC0882311F001501109A5E0B0E007
:108B40000E94C8489B01AC01220F331F441F551FD0
:108B5000280D311D411D511D283999E93907490753
:108B600099E15907A8F2C6609C2ED2CFAEEF8A12C7
:108B700006C0C3FD3CC09C2E689493F8C9CFDF7D2E
:108B8000D534A9F580818D3239F4C061DF011296A8
:108B9000818162E070E006C0DF018B32C1F3119683
:108BA00061E070E080535D01A61AB70A8A30F8F4DC
:108BB000E0E8CE16ECE0DE065CF4B601660F771F47
:108BC000660F771FC60ED71ECC0CDD1CC80ED11C3D
:108BD0005D01FFEFAF1ABF0A8C9180538A30A8F174
:108BE000C4FF03C0D194C194D1080C0D1D1DC1FF59
:108BF00009C0E114F10431F081E0A81AB108D701ED
:108C0000AD92BC92CA01B9010E947147C370C330D2
:108C100009F490584B015C0120E030E0A9010E946A
:108C20006C47882309F440C0CFEED2E017FF05C09F
:108C3000119501951109C7EDD2E06E01B8E1CB1A8B
:108C4000D10880E2E82EF12C0FC0D501B1CFFE0192
:108C500025913591459154910E191F09C501B40113
:108C60000E94D2474B015C01D501C4010E151F05BE
:108C700074F72497F594E794CC16DD06A9F78A2FAC
:108C8000880F8B2F881F8F3F49F020E030E0A9012B
:108C9000C501B4010E946C47811106C082E290E0D8
:108CA0009093D60D8093D50DC501B401DF91CF917E
:108CB0001F910F91FF90EF90DF90CF90BF90AF90FA
:108CC0009F908F900895283008F027E03327DA012D
:108CD000990F311D87FD916000966105710539F48A
:108CE00032602E5F3D9330E32A95E1F708959F3F70
:108CF00030F080387105610509F03C5F3C5F3D93C1
:108D0000913008F08068911DDF93CF931F930F93EC
:108D1000FF92EF92192F987F9695E92F9695969549
:108D2000E90FFF27E35BFC4F99273327EE24FF244D
:108D3000A701E70105900894079428F4360FE71E71
:108D4000F81E491F511D660F771F881F991F069433
:108D5000A1F70590079428F4E70EF81E491F561F47
:108D6000C11D770F881F991F661F0694A1F70590F4
:108D7000079428F4F80E491F561FC71FD11D880FEE
:108D8000991F661F771F0694A1F70590079420F49A
:108D9000490F561FC71FD81F990F661F771F881FBF
:108DA0000694A9F784911095177041F0D695C79550
:108DB00057954795F794E7941A95C1F7E3EFF2E0DA
:108DC00068941590159135916591959105907FE284
:108DD0007395E118F10A430B560BC90BD009C0F784
:108DE000E10CF11E431F561FC91FD01D7EF47033C6
:108DF00011F48A95E6CFE894015030F0080F0AF498
:108E00000027021708F4202F2395022F7A3328F029
:108E100079E37D932A95E9F710C07D932A9589F629
:108E2000069497956795379517951794E118F10A69
:108E3000430B560BC90BD00998F023957E9173957F
:108E40007A3308F070E37C932013B8F77E91706159
:108E50007D9330F0839571E37D9370E32A95E1F77C
:108E60001124EF90FF900F911F91CF91DF919927DF
:108E700087FD9095089591110C943F48803219F028
:108E800089508550C8F70895FB01DC0141505040DE
:108E900088F08D9181341CF08B350CF4805E6591E7
:108EA00061341CF06B350CF4605E861B611171F34C
:108EB000990B0895881BFCCFDC01FC01672F719191
:108EC0007723E1F7329704C07C916D9370836291B0
:108ED000AE17BF07C8F308950E94AE4708F481E0BB
:108EE0000895E89409C097FB3EF49095809570959D
:108EF00061957F4F8F4F9F4F9923A9F0F92F96E9E6
:108F0000BB279395F695879577956795B795F1115A
:108F1000F8CFFAF4BB0F11F460FF1BC06F5F7F4FF7
:108F20008F4F9F4F16C0882311F096E911C0772309
:108F300021F09EE8872F762F05C0662371F096E812
:108F4000862F70E060E02AF09A95660F771F881FE1
:108F5000DAF7880F9695879597F90895990F000885
:108F6000550FAA0BE0E8FEEF16161706E807F907FB
:108F7000C0F012161306E407F50798F0621B730B96
:108F8000840B950B39F40A2661F0232B242B252B17
:108F900021F408950A2609F4A140A6958FEF811DBA
:108FA000811D08950E94E5470C9459480E944B4842
:108FB00038F00E94524820F0952311F00C9442485A
:108FC0000C94484811240C948D480E946A4870F310
:108FD000959FC1F3950F50E0551F629FF001729F5E
:108FE000BB27F00DB11D639FAA27F00DB11DAA1F6D
:108FF000649F6627B00DA11D661F829F2227B00DBA
:10900000A11D621F739FB00DA11D621F839FA00D44
:10901000611D221F749F3327A00D611D231F849F94
:10902000600D211D822F762F6A2F11249F575040EB
:109030009AF0F1F088234AF0EE0FFF1FBB1F661F66
:10904000771F881F91505040A9F79E3F510580F02F
:109050000C9442480C948D485F3FE4F3983ED4F35F
:10906000869577956795B795F795E7959F5FC1F7D3
:10907000FE2B880F911D9695879597F9089599274E
:109080008827089597F99F6780E870E060E0089569
:109090009FEF80EC089500240A9416161706180610
:1090A0000906089500240A941216130614060506EC
:1090B0000895092E0394000C11F4882352F0BB0F7D
:1090C00040F4BF2B11F460FF04C06F5F7F4F8F4FE0
:1090D0009F4F089557FD9058440F551F59F05F3F1B
:1090E00071F04795880F97FB991F61F09F3F79F0CA
:1090F00087950895121613061406551FF2CF46954C
:10910000F1DF08C0161617061806991FF1CF8695CD
:109110007105610508940895E894BB2766277727B1
:10912000CB0197F90895F999FECF92BD81BDF89AC8
:10913000992780B50895262FF999FECF1FBA92BDC1
:1091400081BD20BD0FB6F894FA9AF99A0FBE019628
:109150000895052E97FB1EF400940E94C04857FD09
:1091600007D00E94D34807FC03D04EF40C94C048AB
:1091700050954095309521953F4F4F4F5F4F089543
:1091800090958095709561957F4F8F4F9F4F089573
:109190000E94F548A59F900DB49F900DA49F800D4F
:1091A000911D11240895A1E21A2EAA1BBB1BFD01DB
:1091B0000DC0AA1FBB1FEE1FFF1FA217B307E407B6
:1091C000F50720F0A21BB30BE40BF50B661F771F0E
:1091D000881F991F1A9469F76095709580959095EE
:1091E0009B01AC01BD01CF010895A29FB001B39FC7
:1091F000C001A39F700D811D1124911DB29F700DA0
:10920000811D1124911D08955058BB27AA270E9443
:109210001C490C9459480E944B4838F00E9452480F
:1092200020F039F49F3F19F426F40C9448480EF4CA
:10923000E095E7FB0C944248E92F0E946A4858F3F6
:10924000BA17620773078407950720F079F4A6F52B
:109250000C948C480EF4E0950B2EBA2FA02D0B0128
:10926000B90190010C01CA01A0011124FF27591B6B
:1092700099F0593F50F4503E68F11A16F040A22F71
:10928000232F342F4427585FF3CF469537952795E2
:10929000A795F0405395C9F77EF41F16BA0B620BE1
:1092A000730B840BBAF09150A1F0FF0FBB1F661F28
:1092B000771F881FC2F70EC0BA0F621F731F841F6B
:1092C00048F4879577956795B795F7959E3F08F091
:1092D000B0CF9395880F08F09927EE0F9795879553
:1092E00008950E9485490C9459480E94524858F0AC
:1092F0000E944B4840F029F45F3F29F00C9442480B
:1093000051110C948D480C9448480E946A4868F3A7
:109310009923B1F3552391F3951B550BBB27AA272E
:1093200062177307840738F09F5F5F4F220F331F68
:10933000441FAA1FA9F335D00E2E3AF0E0E832D030
:1093400091505040E695001CCAF72BD0FE2F29D033
:10935000660F771F881FBB1F261737074807AB0705
:10936000B0E809F0BB0B802DBF01FF2793585F4F7A
:109370003AF09E3F510578F00C9442480C948D4889
:109380005F3FE4F3983ED4F3869577956795B7955C
:10939000F7959F5FC9F7880F911D9695879597F967
:1093A0000895E1E0660F771F881FBB1F62177307E0
:1093B0008407BA0720F0621B730B840BBA0BEE1FF5
:1093C00088F7E09508950E94EA496894B1110C94D9
:1093D0008D4808950E94724888F09F5798F0B92FE1
:1093E0009927B751B0F0E1F0660F771F881F991FDA
:1093F0001AF0BA95C9F714C0B13091F00E948C48A8
:10940000B1E008950C948C48672F782F8827B85FB7
:1094100039F0B93FCCF3869577956795B395D9F731
:109420003EF490958095709561957F4F8F4F9F4F3B
:1094300008950E94AE4708F48FEF089597FB072E1A
:1094400016F4009407D077FD09D00E94414A07FC2A
:1094500005D03EF4909581959F4F08957095619544
:109460007F4F0895EE0FFF1F881F8BBF0790F69167
:10947000E02D19940E94F548B7FF0895821B930BC5
:109480000895AA1BBB1B51E107C0AA1FBB1FA6174B
:10949000B70710F0A61BB70B881F991F5A95A9F79D
:1094A00080959095BC01CD0108954F925F926F9287
:1094B0007F928F929F92AF92BF92CF92DF92EF9264
:1094C000FF920F931F93CF93DF938C01009799F432
:1094D000CB01DF91CF911F910F91FF90EF90DF9023
:1094E000CF90BF90AF909F908F907F906F905F9044
:1094F0004F900C941C42FC01E60FF71F9C01225078
:109500003109E217F30708F4AEC0D901CD91DC911F
:109510001197C617D70720F1C530D10578F0CE01D5
:1095200004978617970750F0C61BD70B2297C19355
:10953000D1936D937C93CF010E94B842C801DF9113
:10954000CF911F910F91FF90EF90DF90CF90BF9040
:10955000AF909F908F907F906F905F904F90089505
:109560005B01AC1ABD0A4C018C0E9D1EA091D30D5F
:10957000B091D40D512C412CF12CE12C109731F5E8
:109580008091D10D9091D20D8815990509F05CC09C
:109590004616570608F058C08091F9029091FA02D9
:1095A000009741F48DB79EB74091FD025091FE02A5
:1095B000841B950BE817F90708F055C0F093D20DFE
:1095C000E093D10DF90171836083B8CF8D919C91A7
:1095D000119712966C90129713967C901397A8157A
:1095E000B90559F56C0142E0C40ED11CCA14DB0464
:1095F00020F1AC014A195B09DA011296159780F047
:109600006282738251834083D9016D937C93E1140C
:10961000F10471F0D7011396FC93EE9312978ECF5D
:1096200022968C0F9D1FF90191838083F301EFCF68
:10963000F093D40DE093D30D81CF4816590608F46A
:109640002C017D01D3019ACFCB010E941C427C01E9
:10965000009749F0AE01B8010E94364BC8010E9444
:10966000B84287016BCF10E000E068CFFB01DC015E
:1096700002C001900D9241505040D8F70895FB016F
:10968000DC0101900D920020E1F70895FB01DC015F
:109690004150504048F001900D920020C9F701C0A0
:1096A0001D9241505040E0F708950F931F93CF93C0
:1096B000DF93CDB7DEB72E970FB6F894DEBF0FBE9F
:1096C000CDBF0E891F8986E08C831A8309838FEFB3
:1096D0009FE79E838D83AE01465E5F4F688D798DD7
:1096E000CE0101960E94854B2F813885020F131FF2
:1096F000F80110822E960FB6F894DEBF0FBECDBFD4
:10970000DF91CF911F910F9108952F923F924F9229
:109710005F926F927F928F929F92AF92BF92CF9201
:10972000DF92EF92FF920F931F93CF93DF9300D0BE
:1097300000D000D01F921F92CDB7DEB77C013B0155
:109740008A01FC0117821682838181FFDDC1CE016F
:1097500001965C01F7019381F30193FD859193FFDD
:1097600081913F01882309F453C1853239F493FD77
:10977000859193FF81913F01853229F4B70190E0F3
:109780000E949D4DE7CF912C212C312CFFE1F31548
:1097900038F08B3211F190F4803209F1833229F1E3
:1097A00037FC3CC020ED280F2A3050F536FE20C093
:1097B0008AE0989E200D1124922E06C08D3291F0E1
:1097C000803371F7689430F8F30193FD859193FF2E
:1097D00081913F018111DACF21C0689431F86894FA
:1097E00032F8F2CF689433F8EFCF689434F8ECCFC6
:1097F000EAE02E9E200D1124222E689435F8E4CF45
:109800008E3229F436FC04C1689436F8DDCF8C36EC
:1098100019F4689437F8D8CF8836B1F2982F9F7D25
:1098200095549330E0F08336A1F18337C1F183354D
:1098300009F063C02801F2E04F0E511CF801C0800E
:10984000D180692D70E036FC02C06FEF7FEFC6015A
:109850000E94874D4C01689437F882010AC00C5F62
:109860001F4FFFE3F98388248394912C6501E894CA
:1098700037F833FE2DC0522C8114910471F5552018
:1098800009F468CFB70180E290E00E949D4D5A94A0
:10989000F6CFF801808189830E5F1F4FE4CF280146
:1098A000F2E04F0E511CF801C080D180692D70E0AC
:1098B00036FC02C06FEF7FEFC6010E94924D4C0153
:1098C0008201D5CFB70180E290E00E949D4D2A949D
:1098D0002814190409F0B0F7CECFF60137FC8591B2
:1098E00037FE81916F01B70190E00E949D4D5110AC
:1098F0005A94F1E08F1A9108BFCF843619F0893657
:1099000009F077C0F80137FE6BC0608171818281F8
:1099100093810C5F1F4FF32DFF763F2E97FF09C0F9
:1099200090958095709561957F4F8F4F9F4F68946C
:1099300037F82AE030E0A5010E94CD4DC82ECA18A4
:109940008C2C432C36FE0CC0E89440F8C91440F42B
:1099500034FE05C032FC03C0F32DFE7E4F2E892C51
:1099600044FEAAC0FE01EC0DF11D8081803309F098
:109970009CC0242D297E422E842D8870582E43FCB5
:10998000AAC040FEA4C09C2C821418F42C0C922C6B
:10999000981844FEA6C0B70180E390E00E949D4D58
:1099A00042FE09C088E790E041FE02C088E590E0F1
:1099B000B7010E949D4DC91408F49FC0CA94D12CD0
:1099C0009FEFC91AD90ACA0CDB1CF60182916F01FC
:1099D000B70190E00E949D4DAC14BD04B1F74FCF8C
:1099E00060817181072E000C880B990B0E5F1F4F51
:1099F00092CFD32CE894D4F82AE030E08537E1F117
:109A0000232D297FD22E8F36A9F1F0F4883551F11C
:109A1000F701868197812B960FB6F894DEBF0FBEB3
:109A2000CDBFDF91CF911F910F91FF90EF90DF900D
:109A3000CF90BF90AF909F908F907F906F905F90EE
:109A40004F903F902F900895803749F0883701F765
:109A5000D4FE02C06894D2F820E130E00DC06894D2
:109A6000D4F8F6CF34FE03C0822F8660D82E20E1D2
:109A700032E002C028E030E0F801D7FE0FC060817C
:109A80007181828193810C5F1F4FA5010E94CD4D92
:109A9000C82ECA183D2CE89437F852CF60817181E6
:109AA00090E080E00E5F1F4FF0CF42FC02C0839435
:109AB00063CF8394839460CF842D867809F45CCF40
:109AC000F6CFB70180E290E00E949D4D839482140E
:109AD000C0F3512C5ECF522C5818821408F459CF81
:109AE000F8CF842D867809F466CF8BE241FE80E2C0
:109AF00047FC8DE2B70190E05CCFB70180E390E0D6
:109B00000E949D4D9A9457CF8FEF9FEF84CFFC0119
:109B10000590615070400110D8F7809590958E0F98
:109B20009F1F0895FC016150704001900110D8F70B
:109B3000809590958E0F9F1F08950F931F93CF933D
:109B4000DF93182F092FEB018B8181FD09C01FEFD7
:109B50000FEF812F902FDF91CF911F910F910895DB
:109B600082FF14C02E813F818C819D812817390787
:109B70003CF4E881F981CF010196998388831083B1
:109B80008E819F8101969F838E83E3CFE885F9853F
:109B9000812F1995892BA1F3DACFFA01AA27283052
:109BA00051F1203181F1E8946F936E7F6E5F7F4FAA
:109BB0008F4F9F4FAF4FB1E03ED0B4E03CD0670F26
:109BC000781F891F9A1FA11D680F791F8A1F911D79
:109BD000A11D6A0F711D811D911DA11D20D009F4C9
:109BE00068943F912AE0269F11243019305D31930B
:109BF000DEF6CF010895462F4770405D4193B3E0F4
:109C00000FD0C9F7F6CF462F4F70405D4A3318F09A
:109C1000495D31FD4052419302D0A9F7EACFB4E04B
:109C2000A6959795879577956795BA95C9F7009703
:109C30006105710508959B01AC010A2E06945795A4
:109C4000479537952795BA95C9F7620F731F841FFB
:109C5000951FA01D089512E0C8E9D2E000E006C0FB
:109C6000802FFE010E94324A2196011DC939D10779
:0A9C700080E00807A9F7F894FFCF81
:109C7A001E03191D1D19031E1E0301010101031EE6
:109C8A001F001B1B1B1B001F1F0018181818001F82
:109C9A001F0000000000001F0F1813171713180FDA
:109CAA000F1810101010180F0102000128006F126F
:109CBA00833D1900000000000000000000000000C1
:109CCA00000000000000000000000000000000008A
:109CDA000000000000000100000000000000000079
:109CEA00000000000000000000000000000000006A
:109CFA000000000000000000000100000000000059
:109D0A000000000000000000000000000000000049
:109D1A000000000000000000000000000100000038
:109D2A00440120202020202020202020200028005C
:109D3A003E00A800490009000000010000000000E0
:109D4A000000000000000000000000000000000009
:109D5A0000000000000000000000B44228002800B3
:109D6A0049003E00A8000000000000D70D80000056
:109D7A0000400014005400280049003E00A80000DA
:109D8A00000000B80BB400D007000000000000D0AB
:109D9A0002000000000000000000000000B81E855C
:109DAA003D1F1C1F1E1F1E1F1F1E1F1E1F5E00BCE5
:109DBA00007701000000004A065D05A3059706FE2C
:109DCA0005B205F00500000000340B070B760BDD29
:109DDA000A000BED0ADE0A0000000036115D057666
:109DEA000B4E053031313130313130313130313192
:109DFA003030303030303030303030313030313057
:109E0A0030303030000D0A00526573746F7265206D
:109E1A00454550524F4D00536F6674205265736525
:109E2A007400203D20004F4E004F4646002020205F
:109E3A002020202020202020202020202020202018
:109E4A000025356400475249442020004F555400EC
:109E5A0046616C7365202F200054727565202F208F
:109E6A00002C005377697463682053657474696EB3
:109E7A006773005357446973706C617920200045F9
:109E8A0053503332202020202020005357496E7629
:109E9A00657274657220005357476F6F6477652047
:109EAA002020003534303057202020202020004C3C
:109EBA006F52612054656D702020005357457874A5
:109ECA007261535352200053574869676854656D4D
:109EDA00702000455653656C6563746564200053B1
:109EEA00574E6F54656D702020200053573630420C
:109EFA006F6F7374200053573530426F6F7374005D
:109F0A004578706F72744C696D6974004D61782080
:109F1A0054656D70202020004D696E2054656D7067
:109F2A002020200043757272656E74204320200041
:109F3A002030303030300025303564002D003100BB
:109F4A004348414E47452056414C5545004E4557DA
:109F5A002056414C554500536574202D200056412A
:109F6A00524941424C4520494E50555400574149A7
:109F7A005420464F522054494D4552004F522052C8
:109F8A004541442054484520444F43530054494DC9
:109F9A004552202D3E0054554E494E4720494E50B9
:109FAA0055540053455454494E4753205343524540
:109FBA00454E005741544552204D494E2054454D77
:109FCA0050005741544552204D41582054454D5058
:109FDA0000454C454D454E542053495A4520285773
:109FEA00290054414E4B2053495A4520284C2900F8
:109FFA005246343333205452494747455220285752
:10A00A0029004558504F5254205241544520285750
:10A01A002900464C49434B455220464143544F522E
:10A02A000051554954202F2053415645005245535B
:10A03A00544F52452044454641554C5453003639F5
:10A04A00350050616C6164696E205000506C656126
:10A05A00736520776169740053657474696E67204B
:10A06A00557020537475666600455350333220008C
:10A07A0050696E203135202D3E20004C4F52412030
:10A08A0020004900570041002047656E65726963E8
:10A09A0020496E76657274657200205365636F6E2F
:10A0AA00642053535220416374697665004D696E8A
:10A0BA00203A200043204D6178203A200043005482
:10A0CA00756E652056616C75652023200045787091
:10A0DA006F7274204C696D69742000546573742022
:10A0EA0054656D702050726F62650020402043688D
:10A0FA0065636B2054656D700054656D70205072F5
:10A10A006F6265204661696C656400436865636BCC
:10A11A002026205265736574002A0050616C6164C0
:10A12A00696E2D362000204F4E200041524D2000EE
:10A13A004845414C544820004F274E49474854004F
:10A14A003A007C0050414C4144494E00544F20474C
:10A15A005249440020424F4F53542000544F50203C
:10A16A0055502000454C454D454E54004D415849E7
:10A17A004D554D004E54204D4F44450045584C0016
:10A18A00494D4C005246205445535400544F5055A3
:10A19A00502000544F542000444956455254005808
:10A1AA00464552274400544F50200025303464005D
:10A1BA00534F4C41522000544F54205056002B000C
:10A1CA005E0053454E534F520054756E652320006E
:00000001FF
